 splashscreen

 Timestamp is 1b6e61eb (reproducible build file hash)

 Preferred load address is 10000000

 Start         Length     Name                   Class
 0001:00000000 0001ff81H .text$mn                CODE
 0002:00000000 00000170H .idata$5                DATA
 0002:00000170 00000008H .00cfg                  DATA
 0002:00000178 00000004H .CRT$XCA                DATA
 0002:0000017c 00000004H .CRT$XCZ                DATA
 0002:00000180 00000004H .CRT$XIA                DATA
 0002:00000184 00000004H .CRT$XIZ                DATA
 0002:00000188 00000004H .CRT$XPA                DATA
 0002:0000018c 00000004H .CRT$XPZ                DATA
 0002:00000190 00000004H .CRT$XTA                DATA
 0002:00000194 0000000cH .CRT$XTZ                DATA
 0002:00000198 00000000H .gfids$y                DATA
 0002:000001a0 000089e0H .rdata                  DATA
 0002:00008b80 00000000H .rdata$CastGuardVftablesA DATA
 0002:00008b80 00000000H .rdata$CastGuardVftablesC DATA
 0002:00008b80 00000004H .rdata$sxdata           DATA
 0002:00008b84 000000b8H .rdata$voltmd           DATA
 0002:00008c3c 0000031cH .rdata$zzzdbg           DATA
 0002:00008f58 00000004H .rtc$IAA                DATA
 0002:00008f5c 00000004H .rtc$IZZ                DATA
 0002:00008f60 00000004H .rtc$TAA                DATA
 0002:00008f64 00000004H .rtc$TZZ                DATA
 0002:00008f68 00000084H .xdata$x                DATA
 0002:00008fec 00000020H .didat$2                DATA
 0002:0000900c 00000020H .didat$3                DATA
 0002:0000902c 00000084H .didat$4                DATA
 0002:000090b0 00000204H .didat$6                DATA
 0002:000092b4 0000008cH .didat$7                DATA
 0002:00009340 0000032cH .edata                  DATA
 0002:0000966c 000000dcH .idata$2                DATA
 0002:00009748 00000014H .idata$3                DATA
 0002:0000975c 00000170H .idata$4                DATA
 0002:000098cc 00000690H .idata$6                DATA
 0003:00000000 00000034H .data                   DATA
 0003:00000034 00000084H .didat$5                DATA
 0003:000000b8 00003114H .bss                    DATA
 0004:00000000 00000060H .rsrc$01                DATA
 0004:00000060 00000340H .rsrc$02                DATA

  Address         Publics by Value              Rva+Base       Lib:Object

 0000:00000000       ___AbsoluteZero            00000000     <absolute>
 0000:00000000       ___arm64x_extra_rfe_table  00000000     <absolute>
 0000:00000000       ___arm64x_extra_rfe_table_size 00000000     <absolute>
 0000:00000000       ___arm64x_native_entrypoint 00000000     <absolute>
 0000:00000000       ___arm64x_redirection_metadata 00000000     <absolute>
 0000:00000000       ___arm64x_redirection_metadata_count 00000000     <absolute>
 0000:00000000       ___dynamic_value_reloc_table 00000000     <absolute>
 0000:00000000       ___enclave_config          00000000     <absolute>
 0000:00000000       ___guard_check_icall_a64n_fptr 00000000     <absolute>
 0000:00000000       ___guard_eh_cont_count     00000000     <absolute>
 0000:00000000       ___guard_eh_cont_table     00000000     <absolute>
 0000:00000000       ___guard_fids_count        00000000     <absolute>
 0000:00000000       ___guard_fids_table        00000000     <absolute>
 0000:00000000       ___guard_iat_count         00000000     <absolute>
 0000:00000000       ___guard_iat_table         00000000     <absolute>
 0000:00000000       ___guard_longjmp_count     00000000     <absolute>
 0000:00000000       ___guard_longjmp_table     00000000     <absolute>
 0000:00000000       ___hybrid_auxiliary_delayload_iat 00000000     <absolute>
 0000:00000000       ___hybrid_auxiliary_delayload_iat_copy 00000000     <absolute>
 0000:00000000       ___hybrid_auxiliary_iat    00000000     <absolute>
 0000:00000000       ___hybrid_auxiliary_iat_copy 00000000     <absolute>
 0000:00000000       ___hybrid_code_map         00000000     <absolute>
 0000:00000000       ___hybrid_code_map_count   00000000     <absolute>
 0000:00000000       ___hybrid_image_info_bitfield 00000000     <absolute>
 0000:00000000       ___x64_code_ranges_to_entry_points 00000000     <absolute>
 0000:00000000       ___x64_code_ranges_to_entry_points_count 00000000     <absolute>
 0000:00000001       ___safe_se_handler_count   00000001     <absolute>
 0000:00000100       ___guard_flags             00000100     <absolute>
 0000:00000000       ___ImageBase               10000000     <linker-defined>
 0001:00000f93       _DGifCloseFile             10001f93 f   dgif_lib.obj
 0001:00001324       _DGifDecreaseImageCounter  10002324 f   dgif_lib.obj
 0001:0000135f       _DGifGetCodeNext           1000235f f   dgif_lib.obj
 0001:000013c4       _DGifGetExtension          100023c4 f   dgif_lib.obj
 0001:00001412       _DGifGetExtensionNext      10002412 f   dgif_lib.obj
 0001:00001471       _DGifGetImageDesc          10002471 f   dgif_lib.obj
 0001:00001510       _DGifGetImageHeader        10002510 f   dgif_lib.obj
 0001:00001665       _DGifGetLine               10002665 f   dgif_lib.obj
 0001:0000170e       _DGifGetRecordType         1000270e f   dgif_lib.obj
 0001:00001785       _DGifGetScreenDesc         10002785 f   dgif_lib.obj
 0001:000018f9       _DGifOpen                  100028f9 f   dgif_lib.obj
 0001:00001abc       _DGifSlurp                 10002abc f   dgif_lib.obj
 0001:00001ca4       _GifAddExtensionBlock      10002ca4 f   gifalloc.obj
 0001:00001d1d       _GifBitSize                10002d1d f   gifalloc.obj
 0001:00001d34       _GifFreeExtensions         10002d34 f   gifalloc.obj
 0001:00001d78       _GifFreeMapObject          10002d78 f   gifalloc.obj
 0001:00001d95       _GifFreeSavedImages        10002d95 f   gifalloc.obj
 0001:00001e02       _GifMakeMapObject          10002e02 f   gifalloc.obj
 0001:00001e73       ___local_stdio_printf_options 10002e73 f i gzlib.obj
 0001:00001e79       _inflate_fast              10002e79 f   inffast.obj
 0001:00002281       _inflate                   10003281 f   inflate.obj
 0001:000037ad       _inflateEnd                100047ad f   inflate.obj
 0001:000037ed       _inflateInit2_             100047ed f   inflate.obj
 0001:00003893       _inflateReset              10004893 f   inflate.obj
 0001:000038bc       _inflateReset2             100048bc f   inflate.obj
 0001:00003934       _inflateResetKeep          10004934 f   inflate.obj
 0001:00003aad       _inflate_table             10004aad f   inftrees.obj
 0001:00003ee6       _JNI_OnLoad@8              10004ee6 f   java_awt_SplashScreen.obj
 0001:00003eee       _Java_java_awt_SplashScreen__1close@16 10004eee f   java_awt_SplashScreen.obj
 0001:00003f10       _Java_java_awt_SplashScreen__1getBounds@16 10004f10 f   java_awt_SplashScreen.obj
 0001:00003fe3       _Java_java_awt_SplashScreen__1getImageFileName@16 10004fe3 f   java_awt_SplashScreen.obj
 0001:00004012       _Java_java_awt_SplashScreen__1getImageJarName@16 10005012 f   java_awt_SplashScreen.obj
 0001:00004041       _Java_java_awt_SplashScreen__1getInstance@8 10005041 f   java_awt_SplashScreen.obj
 0001:0000404a       _Java_java_awt_SplashScreen__1getScaleFactor@16 1000504a f   java_awt_SplashScreen.obj
 0001:0000405f       _Java_java_awt_SplashScreen__1isVisible@16 1000505f f   java_awt_SplashScreen.obj
 0001:00004078       _Java_java_awt_SplashScreen__1setImageData@20 10005078 f   java_awt_SplashScreen.obj
 0001:000040d1       _Java_java_awt_SplashScreen__1update@40 100050d1 f   java_awt_SplashScreen.obj
 0001:000041c9       _jAbort                    100051c9 f   jcomapi.obj
 0001:000041fc       _jAlcHTable                100051fc f   jcomapi.obj
 0001:00004218       _jAlcQTable                10005218 f   jcomapi.obj
 0001:00004234       _jDestroy                  10005234 f   jcomapi.obj
 0001:000043b9       _jConsumeInput             100053b9 f   jdapimin.obj
 0001:00004464       _jCreaDecompress           10005464 f   jdapimin.obj
 0001:0000452a       _jDestDecompress           1000552a f   jdapimin.obj
 0001:0000452f       _jFinDecompress            1000552f f   jdapimin.obj
 0001:000045d4       _jReadHeader               100055d4 f   jdapimin.obj
 0001:0000463b       _jReadScanlines            1000563b f   jdapistd.obj
 0001:000046c5       _jStrtDecompress           100056c5 f   jdapistd.obj
 0001:000053f2       ___scrt_stub_for_is_c_termination_complete 100063f2 f   MSVCRT:ucrt_stubs.obj
 0001:000053f2       __is_c_termination_complete 100063f2 f   MSVCRT:ucrt_stubs.obj
 0001:000053f2       _jMemInit                  100063f2 f   jmemnobs.obj
 0001:000053f5       _jIDCoefC                  100063f5 f   jdcoefct.obj
 0001:000057ec       _jIDColor                  100067ec f   jdcolor.obj
 0001:000059d8       @_guard_check_icall_nop@4  100069d8 f   MSVCRT:guard_support.obj
 0001:000059d8       _jMemTerm                  100069d8 f   jmemnobs.obj
 0001:00005c74       _jIIDCT                    10006c74 f   jddctmgr.obj
 0001:00006292       _jFilBitBuf                10007292 f   jdhuff.obj
 0001:0000638a       _jHufDecode                1000738a f   jdhuff.obj
 0001:00006446       _jIHDecoder                10007446 f   jdhuff.obj
 0001:00006485       _jMkDDerived               10007485 f   jdhuff.obj
 0001:00006b5b       _jIInCtlr                  10007b5b f   jdinput.obj
 0001:00006ec4       _jIDMainC                  10007ec4 f   jdmainct.obj
 0001:0000861d       _jIMReader                 1000961d f   jdmarker.obj
 0001:00008689       _jResyncRestart            10009689 f   jdmarker.obj
 0001:00008e51       _jCalcDimensions           10009e51 f   jdmaster.obj
 0001:00009033       _jIDMaster                 1000a033 f   jdmaster.obj
 0001:000098d8       _jIMUpsampler              1000a8d8 f   jdmerge.obj
 0001:0000a396       _jIPHDecoder               1000b396 f   jdphuff.obj
 0001:0000a6cb       _jIDPostC                  1000b6cb f   jdpostct.obj
 0001:0000ad3c       _jIUpsampler               1000bd3c f   jdsample.obj
 0001:0000b02d       __vfprintf_l               1000c02d f i jerror.obj
 0001:0000b09f       _fprintf                   1000c09f f i jerror.obj
 0001:0000b0b7       _jStdError                 1000c0b7 f   jerror.obj
 0001:0000b163       _jRDfloat                  1000c163 f   jidctflt.obj
 0001:0000b60c       _jRDifast                  1000c60c f   jidctfst.obj
 0001:0000b9f6       _jRDislow                  1000c9f6 f   jidctint.obj
 0001:0000bec4       _jRD1x1                    1000cec4 f   jidctred.obj
 0001:0000bf01       _jRD2x2                    1000cf01 f   jidctred.obj
 0001:0000c0c9       _jRD4x4                    1000d0c9 f   jidctred.obj
 0001:0000c3e1       ___local_stdio_scanf_options 1000d3e1 f i jmemmgr.obj
 0001:0000c3e7       __vsscanf_l                1000d3e7 f i jmemmgr.obj
 0001:0000cb56       _jIMemMgr                  1000db56 f   jmemmgr.obj
 0001:0000cefe       _sscanf                    1000defe f i jmemmgr.obj
 0001:0000cf16       _jFreeLarge                1000df16 f   jmemnobs.obj
 0001:0000cf16       _jFreeSmall                1000df16 f   jmemnobs.obj
 0001:0000cf16       _zcfree                    1000df16 f   zutil.obj
 0001:0000cf22       _jGetLarge                 1000df22 f   jmemnobs.obj
 0001:0000cf22       _jGetSmall                 1000df22 f   jmemnobs.obj
 0001:0000cf2e       _jMemAvail                 1000df2e f   jmemnobs.obj
 0001:0000cf48       _jOpenBackStore            1000df48 f   jmemnobs.obj
 0001:0000d486       _jI1Quant                  1000e486 f   jquant1.obj
 0001:0000e1ca       _jI2Quant                  1000f1ca f   jquant2.obj
 0001:0000ee1f       _jCopyBlocks               1000fe1f f   jutils.obj
 0001:0000ee38       _jCopySamples              1000fe38 f   jutils.obj
 0001:0000ee76       _jDivRound                 1000fe76 f   jutils.obj
 0001:0000ee85       _jRound                    1000fe85 f   jutils.obj
 0001:0000ee9c       _jZeroFar                  1000fe9c f   jutils.obj
 0001:0000eeaf       _openbsd_reallocarray      1000feaf f   openbsd-reallocarray.obj
 0001:0000eefe       _png_XYZ_from_xy           1000fefe f   png.obj
 0001:0000f58d       _png_build_gamma_table     1001058d f   png.obj
 0001:0000f71e       _png_calculate_crc         1001071e f   png.obj
 0001:0000f76b       _png_check_IHDR            1001076b f   png.obj
 0001:0000f949       _png_check_fp_number       10010949 f   png.obj
 0001:0000fa88       _png_check_fp_string       10010a88 f   png.obj
 0001:0000fac9       _png_chunk_unknown_handling 10010ac9 f   png.obj
 0001:0000fb16       _png_create_info_struct    10010b16 f   png.obj
 0001:0000fb4a       _png_create_png_struct     10010b4a f   png.obj
 0001:0000fc98       _png_destroy_gamma_table   10010c98 f   png.obj
 0001:0000fdc5       _png_destroy_info_struct   10010dc5 f   png.obj
 0001:0000fe4e       _png_free_data             10010e4e f   png.obj
 0001:000101f9       _png_gamma_16bit_correct   100111f9 f   png.obj
 0001:00010272       _png_gamma_8bit_correct    10011272 f   png.obj
 0001:000102ee       _png_gamma_correct         100112ee f   png.obj
 0001:00010316       _png_gamma_significant     10011316 f   png.obj
 0001:0001032b       _png_get_io_ptr            1001132b f   png.obj
 0001:00010338       _png_handle_as_unknown     10011338 f   png.obj
 0001:00010383       _png_muldiv                10011383 f   png.obj
 0001:0001040b       _png_reciprocal            1001140b f   png.obj
 0001:00010465       _png_reciprocal2           10011465 f   png.obj
 0001:000104dc       _png_reset_crc             100114dc f   png.obj
 0001:000104f4       _png_set_rgb_coefficients  100114f4 f   png.obj
 0001:0001065e       _png_set_sig_bytes         1001165e f   png.obj
 0001:00010689       _png_sig_cmp               10011689 f   png.obj
 0001:000106d2       _png_user_version_check    100116d2 f   png.obj
 0001:000107c4       _png_zalloc                100117c4 f   png.obj
 0001:000107fe       _png_zfree                 100117fe f   png.obj
 0001:00010803       _png_zstream_error         10011803 f   png.obj
 0001:000108bf       _png_app_error             100118bf f   pngerror.obj
 0001:000108df       _png_app_warning           100118df f   pngerror.obj
 0001:000108ff       _png_benign_error          100118ff f   pngerror.obj
 0001:0001095c       _png_chunk_benign_error    1001195c f   pngerror.obj
 0001:0001097c       _png_chunk_error           1001197c f   pngerror.obj
 0001:000109b1       _png_chunk_report          100119b1 f   pngerror.obj
 0001:000109d0       _png_chunk_warning         100119d0 f   pngerror.obj
 0001:00010a64       _png_error                 10011a64 f   pngerror.obj
 0001:00010a88       _png_fixed_error           10011a88 f   pngerror.obj
 0001:00010b87       _png_free_jmpbuf           10011b87 f   pngerror.obj
 0001:00010bfd       _png_longjmp               10011bfd f   pngerror.obj
 0001:00010c23       _png_safecat               10011c23 f   pngerror.obj
 0001:00010c60       _png_set_error_fn          10011c60 f   pngerror.obj
 0001:00010c7e       _png_set_longjmp_fn        10011c7e f   pngerror.obj
 0001:00010cf0       _png_warning               10011cf0 f   pngerror.obj
 0001:00010d50       _png_get_IHDR              10011d50 f   pngget.obj
 0001:00010df5       _png_get_gAMA              10011df5 f   pngget.obj
 0001:00010e31       _png_get_rowbytes          10011e31 f   pngget.obj
 0001:00010e47       _png_calloc                10011e47 f   pngmem.obj
 0001:00010e70       _png_destroy_png_struct    10011e70 f   pngmem.obj
 0001:00010ed4       _png_free                  10011ed4 f   pngmem.obj
 0001:00010efd       _png_malloc                10011efd f   pngmem.obj
 0001:00010f29       _png_malloc_array          10011f29 f   pngmem.obj
 0001:00010f72       _png_malloc_base           10011f72 f   pngmem.obj
 0001:00010f9a       _png_malloc_warn           10011f9a f   pngmem.obj
 0001:00010fc7       _png_realloc_array         10011fc7 f   pngmem.obj
 0001:0001105a       _png_set_mem_fn            1001205a f   pngmem.obj
 0001:00011081       _png_create_read_struct    10012081 f   pngread.obj
 0001:0001109f       _png_create_read_struct_2  1001209f f   pngread.obj
 0001:000110f0       _png_destroy_read_struct   100120f0 f   pngread.obj
 0001:00011300       _png_read_end              10012300 f   pngread.obj
 0001:00011430       _png_read_image            10012430 f   pngread.obj
 0001:000114c7       _png_read_info             100124c7 f   pngread.obj
 0001:000115cc       _png_read_row              100125cc f   pngread.obj
 0001:000118c8       _png_read_update_info      100128c8 f   pngread.obj
 0001:000118fb       _png_start_read_image      100128fb f   pngread.obj
 0001:0001191f       _png_default_read_data     1001291f f   pngrio.obj
 0001:00011952       _png_read_data             10012952 f   pngrio.obj
 0001:00011978       _png_set_read_fn           10012978 f   pngrio.obj
 0001:00013e09       _png_do_read_transformations 10014e09 f   pngrtran.obj
 0001:00014b63       _png_init_read_transformations 10015b63 f   pngrtran.obj
 0001:0001562c       _png_read_transform_info   1001662c f   pngrtran.obj
 0001:000157fc       _png_resolve_file_gamma    100167fc f   pngrtran.obj
 0001:00015871       _png_set_expand            10016871 f   pngrtran.obj
 0001:00015871       _png_set_tRNS_to_alpha     10016871 f   pngrtran.obj
 0001:0001588d       _png_set_expand_gray_1_2_4_to_8 1001688d f   pngrtran.obj
 0001:000158a9       _png_set_gamma             100168a9 f   pngrtran.obj
 0001:000158e9       _png_set_gamma_fixed       100168e9 f   pngrtran.obj
 0001:0001596d       _png_set_gray_to_rgb       1001696d f   pngrtran.obj
 0001:00015990       _png_set_strip_16          10016990 f   pngrtran.obj
 0001:00016f70       _png_combine_row           10017f70 f   pngrutil.obj
 0001:00017428       _png_crc_finish            10018428 f   pngrutil.obj
 0001:000174ef       _png_crc_read              100184ef f   pngrutil.obj
 0001:00017511       _png_do_read_interlace     10018511 f   pngrutil.obj
 0001:00017a0a       _png_get_uint_31           10018a0a f   pngrutil.obj
 0001:00017a46       _png_handle_chunk          10018a46 f   pngrutil.obj
 0001:00017b95       _png_handle_unknown        10018b95 f   pngrutil.obj
 0001:00017db7       _png_read_IDAT_data        10018db7 f   pngrutil.obj
 0001:00017fdd       _png_read_chunk_header     10018fdd f   pngrutil.obj
 0001:000180ad       _png_read_filter_row       100190ad f   pngrutil.obj
 0001:00018350       _png_read_finish_IDAT      10019350 f   pngrutil.obj
 0001:000183a9       _png_read_finish_row       100193a9 f   pngrutil.obj
 0001:0001847c       _png_read_sig              1001947c f   pngrutil.obj
 0001:00018505       _png_read_start_row        10019505 f   pngrutil.obj
 0001:000187c7       _png_zlib_inflate          100197c7 f   pngrutil.obj
 0001:00018860       _png_set_IHDR              10019860 f   pngset.obj
 0001:0001892f       _png_set_PLTE              1001992f f   pngset.obj
 0001:00018a08       _png_set_bKGD              10019a08 f   pngset.obj
 0001:00018a2f       _png_set_cHRM_fixed        10019a2f f   pngset.obj
 0001:00018a8d       _png_set_gAMA_fixed        10019a8d f   pngset.obj
 0001:00018aab       _png_set_hIST              10019aab f   pngset.obj
 0001:00018b35       _png_set_oFFs              10019b35 f   pngset.obj
 0001:00018b60       _png_set_pCAL              10019b60 f   pngset.obj
 0001:00018d76       _png_set_pHYs              10019d76 f   pngset.obj
 0001:00018da1       _png_set_sBIT              10019da1 f   pngset.obj
 0001:00018dc8       _png_set_sCAL_s            10019dc8 f   pngset.obj
 0001:00018f2a       _png_set_sPLT              10019f2a f   pngset.obj
 0001:00019078       _png_set_sRGB              1001a078 f   pngset.obj
 0001:00019099       _png_set_tIME              1001a099 f   pngset.obj
 0001:00019107       _png_set_tRNS              1001a107 f   pngset.obj
 0001:000191f3       _png_set_text_2            1001a1f3 f   pngset.obj
 0001:000194f0       _png_set_unknown_chunks    1001a4f0 f   pngset.obj
 0001:0001961d       _png_do_bgr                1001a61d f   pngtrans.obj
 0001:000196d9       _png_do_check_palette_indexes 1001a6d9 f   pngtrans.obj
 0001:0001980f       _png_do_invert             1001a80f f   pngtrans.obj
 0001:00019879       _png_do_packswap           1001a879 f   pngtrans.obj
 0001:000198be       _png_do_strip_channel      1001a8be f   pngtrans.obj
 0001:00019a08       _png_do_swap               1001aa08 f   pngtrans.obj
 0001:00019a36       _png_set_filler            1001aa36 f   pngtrans.obj
 0001:00019a7f       _png_set_interlace_handling 1001aa7f f   pngtrans.obj
 0001:00019a9c       _blendRGB                  1001aa9c f i splashscreen_gfx_impl.obj
 0001:00019b24       _convertLine               1001ab24 f   splashscreen_gfx_impl.obj
 0001:00019c6b       _convertRect               1001ac6b f   splashscreen_gfx_impl.obj
 0001:00019c82       _convertRect2              1001ac82 f   splashscreen_gfx_impl.obj
 0001:00019d82       _ditherColor               1001ad82 f i splashscreen_gfx_impl.obj
 0001:00019de7       _fillLine                  1001ade7 f i splashscreen_gfx_impl.obj
 0001:00019e1b       _fillRect                  1001ae1b f   splashscreen_gfx_impl.obj
 0001:00019e74       _getMaskShift              1001ae74 f i splashscreen_gfx_impl.obj
 0001:00019ead       _getRGBA                   1001aead f i splashscreen_gfx_impl.obj
 0001:0001a096       _initColorCube             1001b096 f   splashscreen_gfx_impl.obj
 0001:0001a1da       _initDither                1001b1da f   splashscreen_gfx_impl.obj
 0001:0001a23b       _initFormat                1001b23b f   splashscreen_gfx_impl.obj
 0001:0001a2a4       _initRect                  1001b2a4 f   splashscreen_gfx_impl.obj
 0001:0001a2ff       _premultiplyRGBA           1001b2ff f i splashscreen_gfx_impl.obj
 0001:0001a333       _putRGBADither             1001b333 f i splashscreen_gfx_impl.obj
 0001:0001a51a       _quantizeColors            1001b51a f   splashscreen_gfx_impl.obj
 0001:0001a61a       _SplashDecodeGif           1001b61a f   splashscreen_gif.obj
 0001:0001ac40       _SplashDecodeGifStream     1001bc40 f   splashscreen_gif.obj
 0001:0001ac65       _SplashStreamGifInputFunc  1001bc65 f   splashscreen_gif.obj
 0001:0001ac7b       _BitmapToYXBandedRectangles 1001bc7b f   splashscreen_impl.obj
 0001:0001adc9       _GetScaledImageName        1001bdc9 f   splashscreen_impl.obj
 0001:0001b109       _SplashCleanup             1001c109 f   splashscreen_impl.obj
 0001:0001b194       _SplashClose               1001c194 f   splashscreen_impl.obj
 0001:0001b1c3       _SplashDone                1001c1c3 f   splashscreen_impl.obj
 0001:0001b1d2       _SplashGetInstance         1001c1d2 f   splashscreen_impl.obj
 0001:0001b206       _SplashGetScaledImgNameMaxPstfixLen 1001c206 f   splashscreen_impl.obj
 0001:0001b224       _SplashInit                1001c224 f   splashscreen_impl.obj
 0001:0001b275       _SplashIsStillLooping      1001c275 f   splashscreen_impl.obj
 0001:0001b29f       _SplashLoadFile            1001c29f f   splashscreen_impl.obj
 0001:0001b2ce       _SplashLoadMemory          1001c2ce f   splashscreen_impl.obj
 0001:0001b3bd       _SplashNextFrame           1001c3bd f   splashscreen_impl.obj
 0001:0001b439       _SplashSetFileJarName      1001c439 f   splashscreen_impl.obj
 0001:0001b48a       _SplashSetScaleFactor      1001c48a f   splashscreen_impl.obj
 0001:0001b49e       _SplashStart               1001c49e f   splashscreen_impl.obj
 0001:0001b4bf       _SplashStreamInitFile      1001c4bf f   splashscreen_impl.obj
 0001:0001b4f5       _SplashStreamInitMemory    1001c4f5 f   splashscreen_impl.obj
 0001:0001b521       _SplashUpdateScreenData    1001c521 f   splashscreen_impl.obj
 0001:0001b61e       __snprintf                 1001c61e f i splashscreen_impl.obj
 0001:0001b638       __vsnprintf                1001c638 f i splashscreen_impl.obj
 0001:0001b653       __vsnprintf_l              1001c653 f i splashscreen_impl.obj
 0001:0001b686       _cleanUp                   1001c686 f   splashscreen_impl.obj
 0001:0001b74b       _SplashDecodeJpeg          1001c74b f   splashscreen_jpeg.obj
 0001:0001b954       _SplashDecodeJpegStream    1001c954 f   splashscreen_jpeg.obj
 0001:0001bb1c       _SplashDecodePng           1001cb1c f   splashscreen_png.obj
 0001:0001be8a       _SplashDecodePngStream     1001ce8a f   splashscreen_png.obj
 0001:0001bee3       _my_png_read_stream        1001cee3 f   splashscreen_png.obj
 0001:0001bf0f       _SplashCleanupPlatform     1001cf0f f   splashscreen_sys.obj
 0001:0001bf7d       _SplashClosePlatform       1001cf7d f   splashscreen_sys.obj
 0001:0001bf94       _SplashConvertStringAlloc  1001cf94 f   splashscreen_sys.obj
 0001:0001c01c       _SplashCreateThread        1001d01c f   splashscreen_sys.obj
 0001:0001c039       _SplashCreateWindow        1001d039 f   splashscreen_sys.obj
 0001:0001c12c       _SplashDonePlatform        1001d12c f   splashscreen_sys.obj
 0001:0001c142       _SplashGetScaledImageName  1001d142 f   splashscreen_sys.obj
 0001:0001c1aa       _SplashInitFrameShape      1001d1aa f   splashscreen_sys.obj
 0001:0001c31f       _SplashInitPlatform        1001d31f f   splashscreen_sys.obj
 0001:0001c48a       _SplashLock                1001d48a f   splashscreen_sys.obj
 0001:0001c49b       _SplashMessagePump         1001d49b f   splashscreen_sys.obj
 0001:0001c4ce       _SplashPaint               1001d4ce f   splashscreen_sys.obj
 0001:0001c6bc       _SplashReconfigure         1001d6bc f   splashscreen_sys.obj
 0001:0001c6d6       _SplashReconfigureNow      1001d6d6 f   splashscreen_sys.obj
 0001:0001c74f       _SplashRedrawWindow        1001d74f f   splashscreen_sys.obj
 0001:0001c9f1       _SplashScreenThread@4      1001d9f1 f   splashscreen_sys.obj
 0001:0001ca98       _SplashTime                1001da98 f   splashscreen_sys.obj
 0001:0001ca9e       _SplashUnlock              1001da9e f   splashscreen_sys.obj
 0001:0001caaf       _SplashUpdate              1001daaf f   splashscreen_sys.obj
 0001:0001cc55       _GetScreenDpi              1001dc55 f   systemScale.obj
 0001:0001cdcb       _getPrimaryMonitor@0       1001ddcb f   systemScale.obj
 0001:0001cdd8       __tr_flush_bits            1001ddd8 f   trees.obj
 0001:0001cddd       __tr_flush_block           1001dddd f   trees.obj
 0001:0001cfdb       __tr_stored_block          1001dfdb f   trees.obj
 0001:0001e4b4       _adler32                   1001f4b4 f   zadler32.obj
 0001:0001e4b9       _adler32_z                 1001f4b9 f   zadler32.obj
 0001:0001e6f6       _crc32                     1001f6f6 f   zcrc32.obj
 0001:0001e6fb       _crc32_z                   1001f6fb f   zcrc32.obj
 0001:0001e9e4       _zcalloc                   1001f9e4 f   zutil.obj
 0001:0001e9f6       __imp_load__GetMessageA@16 1001f9f6 f   user32:USER32.dll
 0001:0001ea00       __tailMerge_user32_dll     1001fa00     user32:USER32.dll
 0001:0001ea11       __imp_load__TranslateMessage@4 1001fa11 f   user32:USER32.dll
 0001:0001ea1b       __imp_load__DispatchMessageA@4 1001fa1b f   user32:USER32.dll
 0001:0001ea25       __imp_load__PostMessageA@16 1001fa25 f   user32:USER32.dll
 0001:0001ea2f       __imp_load__DefWindowProcA@16 1001fa2f f   user32:USER32.dll
 0001:0001ea39       __imp_load__PostQuitMessage@4 1001fa39 f   user32:USER32.dll
 0001:0001ea43       __imp_load__RegisterClassExA@4 1001fa43 f   user32:USER32.dll
 0001:0001ea4d       __imp_load__CreateWindowExA@48 1001fa4d f   user32:USER32.dll
 0001:0001ea57       __imp_load__DestroyWindow@4 1001fa57 f   user32:USER32.dll
 0001:0001ea61       __imp_load__ShowWindow@8   1001fa61 f   user32:USER32.dll
 0001:0001ea6b       __imp_load__UpdateLayeredWindow@36 1001fa6b f   user32:USER32.dll
 0001:0001ea75       __imp_load__MoveWindow@24  1001fa75 f   user32:USER32.dll
 0001:0001ea7f       __imp_load__IsWindowVisible@4 1001fa7f f   user32:USER32.dll
 0001:0001ea89       __imp_load__SetTimer@16    1001fa89 f   user32:USER32.dll
 0001:0001ea93       __imp_load__KillTimer@8    1001fa93 f   user32:USER32.dll
 0001:0001ea9d       __imp_load__GetSystemMetrics@4 1001fa9d f   user32:USER32.dll
 0001:0001eaa7       __imp_load__UpdateWindow@4 1001faa7 f   user32:USER32.dll
 0001:0001eab1       __imp_load__GetDC@4        1001fab1 f   user32:USER32.dll
 0001:0001eabb       __imp_load__ReleaseDC@8    1001fabb f   user32:USER32.dll
 0001:0001eac5       __imp_load__BeginPaint@8   1001fac5 f   user32:USER32.dll
 0001:0001eacf       __imp_load__EndPaint@8     1001facf f   user32:USER32.dll
 0001:0001ead9       __imp_load__SetWindowRgn@12 1001fad9 f   user32:USER32.dll
 0001:0001eae3       __imp_load__InvalidateRect@12 1001fae3 f   user32:USER32.dll
 0001:0001eaed       __imp_load__GetWindowRect@8 1001faed f   user32:USER32.dll
 0001:0001eaf7       __imp_load__SetCursorPos@8 1001faf7 f   user32:USER32.dll
 0001:0001eb01       __imp_load__SetCursor@4    1001fb01 f   user32:USER32.dll
 0001:0001eb0b       __imp_load__GetCursorPos@4 1001fb0b f   user32:USER32.dll
 0001:0001eb15       __imp_load__WindowFromPoint@8 1001fb15 f   user32:USER32.dll
 0001:0001eb1f       __imp_load__GetWindowLongA@8 1001fb1f f   user32:USER32.dll
 0001:0001eb29       __imp_load__SetWindowLongA@12 1001fb29 f   user32:USER32.dll
 0001:0001eb33       __imp_load__LoadCursorA@8  1001fb33 f   user32:USER32.dll
 0001:0001eb3d       __imp_load__MonitorFromPoint@12 1001fb3d f   user32:USER32.dll
 0001:0001eb47       ?DloadAcquireSectionWriteAccess@@YGXXZ 1001fb47 f i delayimp:delayhlp.obj
 0001:0001eb7a       ?DloadGetSRWLockFunctionPointers@@YGEXZ 1001fb7a f i delayimp:delayhlp.obj
 0001:0001ebf0       ?DloadLock@@YGXXZ          1001fbf0 f i delayimp:delayhlp.obj
 0001:0001ec2f       ?DloadMakePermanentImageCommit@@YGXPAXK@Z 1001fc2f f i delayimp:delayhlp.obj
 0001:0001ec9e       ?DloadObtainSection@@YGPAXPAK0@Z 1001fc9e f i delayimp:delayhlp.obj
 0001:0001ed19       ?DloadProtectSection@@YGXKPAK@Z 1001fd19 f i delayimp:delayhlp.obj
 0001:0001ed87       ?DloadReleaseSectionWriteAccess@@YGXXZ 1001fd87 f i delayimp:delayhlp.obj
 0001:0001edbd       ?DloadUnlock@@YGXXZ        1001fdbd f i delayimp:delayhlp.obj
 0001:0001ede9       ___delayLoadHelper2@8      1001fde9 f   delayimp:delayhlp.obj
 0001:0001f058       _JDK_LoadSystemLibrary     10020058 f   java:java.dll
 0001:0001f05e       @__security_check_cookie@4 1002005e f   MSVCRT:secchk.obj
 0001:0001f06c       ___raise_securityfailure   1002006c f   MSVCRT:gs_report.obj
 0001:0001f094       ___report_gsfailure        10020094 f   MSVCRT:gs_report.obj
 0001:0001f18e       ___report_rangecheckfailure 1002018e f   MSVCRT:gs_report.obj
 0001:0001f19a       ___report_securityfailure  1002019a f   MSVCRT:gs_report.obj
 0001:0001f270       __ftol2                    10020270 f   MSVCRT:ftol2.obj
 0001:0001f320       __alloca_probe_16          10020320 f   MSVCRT:alloca16.obj
 0001:0001f336       __alloca_probe_8           10020336     MSVCRT:alloca16.obj
 0001:0001f690       __DllMainCRTStartup@12     10020690 f   MSVCRT:dll_dllmain.obj
 0001:0001f6b3       ___isa_available_init      100206b3 f   MSVCRT:cpu_disp.obj
 0001:0001f890       __alloca_probe             10020890 f   MSVCRT:chkstk.obj
 0001:0001f890       __chkstk                   10020890 f   MSVCRT:chkstk.obj
 0001:0001f908       ___security_init_cookie    10020908 f   MSVCRT:gs_support.obj
 0001:0001f953       _DllMain@12                10020953 f   MSVCRT:dll_dllmain_stub.obj
 0001:0001f975       ?__scrt_initialize_type_info@@YAXXZ 10020975 f   MSVCRT:tncleanup.obj
 0001:0001f981       ?__scrt_uninitialize_type_info@@YAXXZ 10020981 f   MSVCRT:tncleanup.obj
 0001:0001f98d       ___scrt_initialize_default_local_stdio_options 1002098d f   MSVCRT:default_local_stdio_options.obj
 0001:0001f9ee       ___scrt_acquire_startup_lock 100209ee f   MSVCRT:utility.obj
 0001:0001fa20       ___scrt_dllmain_after_initialize_c 10020a20 f   MSVCRT:utility.obj
 0001:0001fa4b       ___scrt_dllmain_before_initialize_c 10020a4b f   MSVCRT:utility.obj
 0001:0001fa59       ___scrt_dllmain_crt_thread_attach 10020a59 f   MSVCRT:utility.obj
 0001:0001fa78       ___scrt_dllmain_crt_thread_detach 10020a78 f   MSVCRT:utility.obj
 0001:0001fa85       ___scrt_dllmain_exception_filter 10020a85 f   MSVCRT:utility.obj
 0001:0001fab9       ___scrt_dllmain_uninitialize_c 10020ab9 f   MSVCRT:utility.obj
 0001:0001fadc       ___scrt_dllmain_uninitialize_critical 10020adc f   MSVCRT:utility.obj
 0001:0001fae9       ___scrt_initialize_crt     10020ae9 f   MSVCRT:utility.obj
 0001:0001fb22       ___scrt_initialize_onexit_tables 10020b22 f   MSVCRT:utility.obj
 0001:0001fba9       ___scrt_is_nonwritable_in_current_image 10020ba9 f   MSVCRT:utility.obj
 0001:0001fc3d       ___scrt_release_startup_lock 10020c3d f   MSVCRT:utility.obj
 0001:0001fc5a       ___scrt_uninitialize_crt   10020c5a f   MSVCRT:utility.obj
 0001:0001fc82       ___scrt_get_dyn_tls_init_callback 10020c82 f   MSVCRT:dyn_tls_init.obj
 0001:0001fc88       ___scrt_fastfail           10020c88 f   MSVCRT:utility_desktop.obj
 0001:0001fda3       __crt_debugger_hook        10020da3 f   MSVCRT:utility_desktop.obj
 0001:0001fdab       __RTC_Initialize           10020dab f   MSVCRT:initsect.obj
 0001:0001fdd7       __RTC_Terminate            10020dd7 f   MSVCRT:initsect.obj
 0001:0001fe10       __SEH_prolog4              10020e10 f   MSVCRT:sehprolg4.obj
 0001:0001fe55       __except_handler4          10020e55 f   MSVCRT:chandler4gs.obj
 0001:0001fe84       __get_startup_argv_mode    10020e84 f   MSVCRT:argv_mode.obj
 0001:0001fe88       ___scrt_is_ucrt_dll_in_use 10020e88 f   MSVCRT:ucrt_detection.obj
 0001:0001fe94       _memcpy                    10020e94 f   vcruntime:VCRUNTIME140.dll
 0001:0001fe9a       _memset                    10020e9a f   vcruntime:VCRUNTIME140.dll
 0001:0001fea0       _memcmp                    10020ea0 f   vcruntime:VCRUNTIME140.dll
 0001:0001fea6       _longjmp                   10020ea6 f   vcruntime:VCRUNTIME140.dll
 0001:0001feac       __setjmp3                  10020eac f   vcruntime:VCRUNTIME140.dll
 0001:0001feb2       _strrchr                   10020eb2 f   vcruntime:VCRUNTIME140.dll
 0001:0001feb8       ___std_type_info_destroy_list 10020eb8 f   vcruntime:VCRUNTIME140.dll
 0001:0001febe       __except_handler4_common   10020ebe f   vcruntime:VCRUNTIME140.dll
 0001:0001fec4       _strlen                    10020ec4 f   ucrt:api-ms-win-crt-string-l1-1-0.dll
 0001:0001feca       _pow                       10020eca f   ucrt:api-ms-win-crt-math-l1-1-0.dll
 0001:0001fed0       _strcpy                    10020ed0 f   ucrt:api-ms-win-crt-string-l1-1-0.dll
 0001:0001fed6       __initterm                 10020ed6 f   ucrt:api-ms-win-crt-runtime-l1-1-0.dll
 0001:0001fedc       __initterm_e               10020edc f   ucrt:api-ms-win-crt-runtime-l1-1-0.dll
 0001:0001fee2       __seh_filter_dll           10020ee2 f   ucrt:api-ms-win-crt-runtime-l1-1-0.dll
 0001:0001fee8       __configure_narrow_argv    10020ee8 f   ucrt:api-ms-win-crt-runtime-l1-1-0.dll
 0001:0001feee       __initialize_narrow_environment 10020eee f   ucrt:api-ms-win-crt-runtime-l1-1-0.dll
 0001:0001fef4       __initialize_onexit_table  10020ef4 f   ucrt:api-ms-win-crt-runtime-l1-1-0.dll
 0001:0001fefa       __execute_onexit_table     10020efa f   ucrt:api-ms-win-crt-runtime-l1-1-0.dll
 0001:0001ff00       __cexit                    10020f00 f   ucrt:api-ms-win-crt-runtime-l1-1-0.dll
 0001:0001ff06       ___acrt_initialize         10020f06 f   MSVCRT:ucrt_stubs.obj
 0001:0001ff06       ___acrt_thread_attach      10020f06 f   MSVCRT:ucrt_stubs.obj
 0001:0001ff06       ___acrt_thread_detach      10020f06 f   MSVCRT:ucrt_stubs.obj
 0001:0001ff06       ___acrt_uninitialize       10020f06 f   MSVCRT:ucrt_stubs.obj
 0001:0001ff06       ___acrt_uninitialize_critical 10020f06 f   MSVCRT:ucrt_stubs.obj
 0001:0001ff06       ___scrt_stub_for_acrt_initialize 10020f06 f   MSVCRT:ucrt_stubs.obj
 0001:0001ff06       ___scrt_stub_for_acrt_thread_attach 10020f06 f   MSVCRT:ucrt_stubs.obj
 0001:0001ff06       ___scrt_stub_for_acrt_thread_detach 10020f06 f   MSVCRT:ucrt_stubs.obj
 0001:0001ff06       ___scrt_stub_for_acrt_uninitialize 10020f06 f   MSVCRT:ucrt_stubs.obj
 0001:0001ff06       ___scrt_stub_for_acrt_uninitialize_critical 10020f06 f   MSVCRT:ucrt_stubs.obj
 0001:0001ff06       ___vcrt_initialize         10020f06 f   MSVCRT:ucrt_stubs.obj
 0001:0001ff06       ___vcrt_thread_attach      10020f06 f   MSVCRT:ucrt_stubs.obj
 0001:0001ff06       ___vcrt_thread_detach      10020f06 f   MSVCRT:ucrt_stubs.obj
 0001:0001ff06       ___vcrt_uninitialize       10020f06 f   MSVCRT:ucrt_stubs.obj
 0001:0001ff06       ___vcrt_uninitialize_critical 10020f06 f   MSVCRT:ucrt_stubs.obj
 0001:0001ff09       __filter_x86_sse2_floating_point_exception 10020f09 f   MSVCRT:x86_exception_filter.obj
 0001:0001ff09       __filter_x86_sse2_floating_point_exception_default 10020f09 f   MSVCRT:x86_exception_filter.obj
 0002:00000000       __imp__CreatePalette@4     10021000     gdi32:GDI32.dll
 0002:00000004       __imp__CreateDIBSection@24 10021004     gdi32:GDI32.dll
 0002:00000008       __imp__StretchDIBits@52    10021008     gdi32:GDI32.dll
 0002:0000000c       __imp__SelectPalette@12    1002100c     gdi32:GDI32.dll
 0002:00000010       __imp__SelectObject@8      10021010     gdi32:GDI32.dll
 0002:00000014       __imp__RealizePalette@4    10021014     gdi32:GDI32.dll
 0002:00000018       __imp__GetDeviceCaps@8     10021018     gdi32:GDI32.dll
 0002:0000001c       __imp__ExtCreateRegion@12  1002101c     gdi32:GDI32.dll
 0002:00000020       __imp__DeleteObject@4      10021020     gdi32:GDI32.dll
 0002:00000024       __imp__CombineRgn@16       10021024     gdi32:GDI32.dll
 0002:00000028       __imp__CreateCompatibleDC@4 10021028     gdi32:GDI32.dll
 0002:0000002c       __imp__CreateRectRgn@16    1002102c     gdi32:GDI32.dll
 0002:00000030       __imp__DeleteDC@4          10021030     gdi32:GDI32.dll
 0002:00000034       \177GDI32_NULL_THUNK_DATA  10021034     gdi32:GDI32.dll
 0002:00000038       __imp__IsDebuggerPresent@0 10021038     kernel32:KERNEL32.dll
 0002:0000003c       __imp__GetProcAddress@8    1002103c     kernel32:KERNEL32.dll
 0002:00000040       __imp__MultiByteToWideChar@24 10021040     kernel32:KERNEL32.dll
 0002:00000044       __imp__GetModuleHandleA@4  10021044     kernel32:KERNEL32.dll
 0002:00000048       __imp__GetTickCount@0      10021048     kernel32:KERNEL32.dll
 0002:0000004c       __imp__CreateThread@24     1002104c     kernel32:KERNEL32.dll
 0002:00000050       __imp__LeaveCriticalSection@4 10021050     kernel32:KERNEL32.dll
 0002:00000054       __imp__EnterCriticalSection@4 10021054     kernel32:KERNEL32.dll
 0002:00000058       __imp__InitializeCriticalSection@4 10021058     kernel32:KERNEL32.dll
 0002:0000005c       __imp__InitializeSListHead@4 1002105c     kernel32:KERNEL32.dll
 0002:00000060       __imp__DisableThreadLibraryCalls@4 10021060     kernel32:KERNEL32.dll
 0002:00000064       __imp__GetSystemTimeAsFileTime@4 10021064     kernel32:KERNEL32.dll
 0002:00000068       __imp__GetCurrentThreadId@0 10021068     kernel32:KERNEL32.dll
 0002:0000006c       __imp__GetCurrentProcessId@0 1002106c     kernel32:KERNEL32.dll
 0002:00000070       __imp__QueryPerformanceCounter@4 10021070     kernel32:KERNEL32.dll
 0002:00000074       __imp__IsProcessorFeaturePresent@4 10021074     kernel32:KERNEL32.dll
 0002:00000078       __imp__TerminateProcess@8  10021078     kernel32:KERNEL32.dll
 0002:0000007c       __imp__GetCurrentProcess@0 1002107c     kernel32:KERNEL32.dll
 0002:00000080       __imp__SetUnhandledExceptionFilter@4 10021080     kernel32:KERNEL32.dll
 0002:00000084       __imp__UnhandledExceptionFilter@4 10021084     kernel32:KERNEL32.dll
 0002:00000088       __imp__LoadLibraryExA@12   10021088     kernel32:KERNEL32.dll
 0002:0000008c       __imp__GetModuleHandleW@4  1002108c     kernel32:KERNEL32.dll
 0002:00000090       __imp__FreeLibrary@4       10021090     kernel32:KERNEL32.dll
 0002:00000094       __imp__VirtualQuery@12     10021094     kernel32:KERNEL32.dll
 0002:00000098       __imp__VirtualProtect@16   10021098     kernel32:KERNEL32.dll
 0002:0000009c       __imp__GetSystemInfo@4     1002109c     kernel32:KERNEL32.dll
 0002:000000a0       __imp__GetLastError@0      100210a0     kernel32:KERNEL32.dll
 0002:000000a4       __imp__RaiseException@16   100210a4     kernel32:KERNEL32.dll
 0002:000000a8       \177KERNEL32_NULL_THUNK_DATA 100210a8     kernel32:KERNEL32.dll
 0002:000000ac       __imp__memcpy              100210ac     vcruntime:VCRUNTIME140.dll
 0002:000000b0       __imp__memset              100210b0     vcruntime:VCRUNTIME140.dll
 0002:000000b4       __imp__memcmp              100210b4     vcruntime:VCRUNTIME140.dll
 0002:000000b8       __imp____std_type_info_destroy_list 100210b8     vcruntime:VCRUNTIME140.dll
 0002:000000bc       __imp__strrchr             100210bc     vcruntime:VCRUNTIME140.dll
 0002:000000c0       __imp__longjmp             100210c0     vcruntime:VCRUNTIME140.dll
 0002:000000c4       __imp___setjmp3            100210c4     vcruntime:VCRUNTIME140.dll
 0002:000000c8       __imp___except_handler4_common 100210c8     vcruntime:VCRUNTIME140.dll
 0002:000000cc       \177VCRUNTIME140_NULL_THUNK_DATA 100210cc     vcruntime:VCRUNTIME140.dll
 0002:000000d0       __imp__strtod              100210d0     ucrt:api-ms-win-crt-convert-l1-1-0.dll
 0002:000000d4       \177api-ms-win-crt-convert-l1-1-0_NULL_THUNK_DATA 100210d4     ucrt:api-ms-win-crt-convert-l1-1-0.dll
 0002:000000d8       __imp__getenv              100210d8     ucrt:api-ms-win-crt-environment-l1-1-0.dll
 0002:000000dc       \177api-ms-win-crt-environment-l1-1-0_NULL_THUNK_DATA 100210dc     ucrt:api-ms-win-crt-environment-l1-1-0.dll
 0002:000000e0       __imp__free                100210e0     ucrt:api-ms-win-crt-heap-l1-1-0.dll
 0002:000000e4       __imp__realloc             100210e4     ucrt:api-ms-win-crt-heap-l1-1-0.dll
 0002:000000e8       __imp__malloc              100210e8     ucrt:api-ms-win-crt-heap-l1-1-0.dll
 0002:000000ec       __imp__calloc              100210ec     ucrt:api-ms-win-crt-heap-l1-1-0.dll
 0002:000000f0       \177api-ms-win-crt-heap-l1-1-0_NULL_THUNK_DATA 100210f0     ucrt:api-ms-win-crt-heap-l1-1-0.dll
 0002:000000f4       __imp__pow                 100210f4     ucrt:api-ms-win-crt-math-l1-1-0.dll
 0002:000000f8       __imp__floor               100210f8     ucrt:api-ms-win-crt-math-l1-1-0.dll
 0002:000000fc       \177api-ms-win-crt-math-l1-1-0_NULL_THUNK_DATA 100210fc     ucrt:api-ms-win-crt-math-l1-1-0.dll
 0002:00000100       __imp___initialize_onexit_table 10021100     ucrt:api-ms-win-crt-runtime-l1-1-0.dll
 0002:00000104       __imp___initialize_narrow_environment 10021104     ucrt:api-ms-win-crt-runtime-l1-1-0.dll
 0002:00000108       __imp___cexit              10021108     ucrt:api-ms-win-crt-runtime-l1-1-0.dll
 0002:0000010c       __imp___configure_narrow_argv 1002110c     ucrt:api-ms-win-crt-runtime-l1-1-0.dll
 0002:00000110       __imp___seh_filter_dll     10021110     ucrt:api-ms-win-crt-runtime-l1-1-0.dll
 0002:00000114       __imp___initterm_e         10021114     ucrt:api-ms-win-crt-runtime-l1-1-0.dll
 0002:00000118       __imp___initterm           10021118     ucrt:api-ms-win-crt-runtime-l1-1-0.dll
 0002:0000011c       __imp___execute_onexit_table 1002111c     ucrt:api-ms-win-crt-runtime-l1-1-0.dll
 0002:00000120       __imp___errno              10021120     ucrt:api-ms-win-crt-runtime-l1-1-0.dll
 0002:00000124       __imp__abort               10021124     ucrt:api-ms-win-crt-runtime-l1-1-0.dll
 0002:00000128       \177api-ms-win-crt-runtime-l1-1-0_NULL_THUNK_DATA 10021128     ucrt:api-ms-win-crt-runtime-l1-1-0.dll
 0002:0000012c       __imp____acrt_iob_func     1002112c     ucrt:api-ms-win-crt-stdio-l1-1-0.dll
 0002:00000130       __imp__fread               10021130     ucrt:api-ms-win-crt-stdio-l1-1-0.dll
 0002:00000134       __imp__fclose              10021134     ucrt:api-ms-win-crt-stdio-l1-1-0.dll
 0002:00000138       __imp__ungetc              10021138     ucrt:api-ms-win-crt-stdio-l1-1-0.dll
 0002:0000013c       __imp__fgetc               1002113c     ucrt:api-ms-win-crt-stdio-l1-1-0.dll
 0002:00000140       __imp____stdio_common_vfprintf 10021140     ucrt:api-ms-win-crt-stdio-l1-1-0.dll
 0002:00000144       __imp____stdio_common_vsprintf 10021144     ucrt:api-ms-win-crt-stdio-l1-1-0.dll
 0002:00000148       __imp__fopen               10021148     ucrt:api-ms-win-crt-stdio-l1-1-0.dll
 0002:0000014c       __imp____stdio_common_vsscanf 1002114c     ucrt:api-ms-win-crt-stdio-l1-1-0.dll
 0002:00000150       \177api-ms-win-crt-stdio-l1-1-0_NULL_THUNK_DATA 10021150     ucrt:api-ms-win-crt-stdio-l1-1-0.dll
 0002:00000154       __imp___strdup             10021154     ucrt:api-ms-win-crt-string-l1-1-0.dll
 0002:00000154       __imp__strdup              10021154     ucrt:api-ms-win-crt-string-l1-1-0.dll
 0002:00000158       __imp__strcpy              10021158     ucrt:api-ms-win-crt-string-l1-1-0.dll
 0002:0000015c       __imp__strncmp             1002115c     ucrt:api-ms-win-crt-string-l1-1-0.dll
 0002:00000160       __imp__strlen              10021160     ucrt:api-ms-win-crt-string-l1-1-0.dll
 0002:00000164       \177api-ms-win-crt-string-l1-1-0_NULL_THUNK_DATA 10021164     ucrt:api-ms-win-crt-string-l1-1-0.dll
 0002:00000168       __imp__JDK_LoadSystemLibrary 10021168     java:java.dll
 0002:0000016c       \177java_NULL_THUNK_DATA   1002116c     java:java.dll
 0002:00000170       ___guard_check_icall_fptr  10021170     MSVCRT:guard_support.obj
 0002:00000174       ___castguard_check_failure_os_handled_fptr 10021174     MSVCRT:guard_support.obj
 0002:00000178       ___xc_a                    10021178     MSVCRT:initializers.obj
 0002:0000017c       ___xc_z                    1002117c     MSVCRT:initializers.obj
 0002:00000180       ___xi_a                    10021180     MSVCRT:initializers.obj
 0002:00000184       ___xi_z                    10021184     MSVCRT:initializers.obj
 0002:00000188       ___xp_a                    10021188     MSVCRT:initializers.obj
 0002:0000018c       ___xp_z                    1002118c     MSVCRT:initializers.obj
 0002:00000190       ___xt_a                    10021190     MSVCRT:initializers.obj
 0002:00000194       ___xt_z                    10021194     MSVCRT:initializers.obj
 0002:000001a0       ??_C@_05OJPKCACG@1?43?41@  100211a0     compress.obj
 0002:000001a8       _deflate_copyright         100211a8     deflate.obj
 0002:000002ac       ??_C@_02JDPG@rb@           100212ac     dgif_lib.obj
 0002:000002b0       ??_C@_06MGBLNLI@GIFVER@    100212b0     dgif_lib.obj
 0002:000002b8       ??_C@_0O@BNNCBLEN@out?5of?5memory@ 100212b8     gzlib.obj
 0002:000002c6       ??_C@_00CNPNBAHC@@         100212c6     gzlib.obj
 0002:00000b70       ??_C@_0BD@PJCBIDD@invalid?5block?5type@ 10021b70     infback.obj
 0002:00000b84       ??_C@_0BN@LGAADGOK@invalid?5stored?5block?5lengths@ 10021b84     infback.obj
 0002:00000ba4       ??_C@_0CE@GMIGFPBB@too?5many?5length?5or?5distance?5sym@ 10021ba4     infback.obj
 0002:00000bc8       ??_C@_0BJ@HDEPPGOH@invalid?5code?5lengths?5set@ 10021bc8     infback.obj
 0002:00000be4       ??_C@_0BK@BMMPFBBH@invalid?5bit?5length?5repeat@ 10021be4     infback.obj
 0002:00000c00       ??_C@_0CF@DGDMADCD@invalid?5code?5?9?9?5missing?5end?9of?9@ 10021c00     infback.obj
 0002:00000c28       ??_C@_0BM@IIMGAINC@invalid?5literal?1lengths?5set@ 10021c28     infback.obj
 0002:00000c44       ??_C@_0BG@GMDFCBGP@invalid?5distances?5set@ 10021c44     infback.obj
 0002:00000c5c       ??_C@_0BM@FFFLPBBC@invalid?5literal?1length?5code@ 10021c5c     infback.obj
 0002:00000c78       ??_C@_0BG@LBKINIKP@invalid?5distance?5code@ 10021c78     infback.obj
 0002:00000c90       ??_C@_0BO@ECPMAOGG@invalid?5distance?5too?5far?5back@ 10021c90     infback.obj
 0002:00001558       ??_C@_0BH@LIBMMIGA@incorrect?5header?5check@ 10022558     inflate.obj
 0002:00001570       ??_C@_0BL@IHKGDAEE@unknown?5compression?5method@ 10022570     inflate.obj
 0002:0000158c       ??_C@_0BE@EMOGCLGO@invalid?5window?5size@ 1002258c     inflate.obj
 0002:000015a0       ??_C@_0BJ@BLBBCOMO@unknown?5header?5flags?5set@ 100225a0     inflate.obj
 0002:000015bc       ??_C@_0BE@GONKLEPM@header?5crc?5mismatch@ 100225bc     inflate.obj
 0002:000015d0       ??_C@_0BF@MEIGEHBE@incorrect?5data?5check@ 100225d0     inflate.obj
 0002:000015e8       ??_C@_0BH@FGKKJGOC@incorrect?5length?5check@ 100225e8     inflate.obj
 0002:00001600       _inflate_copyright         10022600     inftrees.obj
 0002:00001730       ??_C@_0BD@KACEDCCP@java?1awt?1Rectangle@ 10022730     java_awt_SplashScreen.obj
 0002:00001744       ??_C@_07CBAIJIEJ@?$CIIIII?$CJV@ 10022744     java_awt_SplashScreen.obj
 0002:0000174c       ??_C@_06FALKBLGB@?$DMinit?$DO@ 1002274c     java_awt_SplashScreen.obj
 0002:00001754       __real@3f800000            10022754     java_awt_SplashScreen.obj
 0002:00001758       __real@3ff0000000000000    10022758     jcapimin.obj
 0002:00001d98       _jMsgTable                 10022d98     jerror.obj
 0002:00001f8c       ??_C@_0BG@MIBALFBH@Bogus?5message?5code?5?$CFd@ 10022f8c     jerror.obj
 0002:00001fa4       ??_C@_0DJ@KONAFFHE@Sorry?0?5there?5are?5legal?5restrict@ 10022fa4     jerror.obj
 0002:00001fe0       ??_C@_0CA@FDMPGPNI@ALIGN_TYPE?5is?5wrong?0?5please?5fix@ 10022fe0     jerror.obj
 0002:00002000       ??_C@_0CF@DENLILGA@MAX_ALLOC_CHUNK?5is?5wrong?0?5pleas@ 10023000     jerror.obj
 0002:00002028       ??_C@_0BK@DKALDNKG@Bogus?5buffer?5control?5mode@ 10023028     jerror.obj
 0002:00002044       ??_C@_0BP@ONFLCDHG@Invalid?5component?5ID?5?$CFd?5in?5SOS@ 10023044     jerror.obj
 0002:00002064       ??_C@_0BN@OJEJKKDL@DCT?5coefficient?5out?5of?5range@ 10023064     jerror.obj
 0002:00002084       ??_C@_0CI@MBJANLAP@IDCT?5output?5block?5size?5?$CFd?5not?5s@ 10023084     jerror.obj
 0002:000020ac       ??_C@_0BP@EOFJNLFD@Bogus?5Huffman?5table?5definition@ 100230ac     jerror.obj
 0002:000020cc       ??_C@_0BH@BGDIGLHC@Bogus?5input?5colorspace@ 100230cc     jerror.obj
 0002:000020e4       ??_C@_0BG@NEGIHEMC@Bogus?5JPEG?5colorspace@ 100230e4     jerror.obj
 0002:000020fc       ??_C@_0BE@OGLAEMOG@Bogus?5marker?5length@ 100230fc     jerror.obj
 0002:00002110       ??_C@_0DN@ELFKFKL@Wrong?5JPEG?5library?5version?3?5lib@ 10023110     jerror.obj
 0002:00002150       ??_C@_0DA@HLEOHNPA@Sampling?5factors?5too?5large?5for?5@ 10023150     jerror.obj
 0002:00002180       ??_C@_0BM@OEMICEFD@Invalid?5memory?5pool?5code?5?$CFd@ 10023180     jerror.obj
 0002:0000219c       ??_C@_0CD@LDBDNLHK@Unsupported?5JPEG?5data?5precision@ 1002319c     jerror.obj
 0002:000021c0       ??_C@_0DH@LNGGEGOL@Invalid?5progressive?5parameters?5@ 100231c0     jerror.obj
 0002:000021f8       ??_C@_0DH@HIKEGPKP@Invalid?5progressive?5parameters?5@ 100231f8     jerror.obj
 0002:00002230       ??_C@_0BH@HMMHPOPE@Bogus?5sampling?5factors@ 10023230     jerror.obj
 0002:00002248       ??_C@_0CA@MJDDICLK@Invalid?5scan?5script?5at?5entry?5?$CFd@ 10023248     jerror.obj
 0002:00002268       ??_C@_0CK@BAMFIBMM@Improper?5call?5to?5JPEG?5library?5i@ 10023268     jerror.obj
 0002:00002298       ??_C@_0EN@DKAEGIBH@JPEG?5parameter?5struct?5mismatch?3@ 10023298     jerror.obj
 0002:000022e8       ??_C@_0BL@CBOEEPLK@Bogus?5virtual?5array?5access@ 100232e8     jerror.obj
 0002:00002304       ??_C@_0CL@JKHIPJLJ@Buffer?5passed?5to?5JPEG?5library?5i@ 10023304     jerror.obj
 0002:00002330       ??_C@_0BM@PKHCPJDH@Suspension?5not?5allowed?5here@ 10023330     jerror.obj
 0002:0000234c       ??_C@_0CF@LAEFHNAH@CCIR601?5sampling?5not?5implemente@ 1002334c     jerror.obj
 0002:00002374       ??_C@_0CG@BEBDNOCG@Too?5many?5color?5components?3?5?$CFd?0?5@ 10023374     jerror.obj
 0002:0000239c       ??_C@_0CF@JDLOPNGO@Unsupported?5color?5conversion?5re@ 1002339c     jerror.obj
 0002:000023c4       ??_C@_0BD@LDBBBMFL@Bogus?5DAC?5index?5?$CFd@ 100233c4     jerror.obj
 0002:000023d8       ??_C@_0BF@CLIOOJFM@Bogus?5DAC?5value?50x?$CFx@ 100233d8     jerror.obj
 0002:000023f0       ??_C@_0BD@KJHFPHIC@Bogus?5DHT?5index?5?$CFd@ 100233f0     jerror.obj
 0002:00002404       ??_C@_0BD@DIMECAOP@Bogus?5DQT?5index?5?$CFd@ 10023404     jerror.obj
 0002:00002418       ??_C@_0CF@DAGGEAPM@Empty?5JPEG?5image?5?$CIDNL?5not?5suppo@ 10023418     jerror.obj
 0002:00002440       ??_C@_0BF@CPNENPBA@Read?5from?5EMS?5failed@ 10023440     jerror.obj
 0002:00002458       ??_C@_0BE@DGJBKIEB@Write?5to?5EMS?5failed@ 10023458     jerror.obj
 0002:0000246c       ??_C@_0CB@DMGINPNE@Didn?8t?5expect?5more?5than?5one?5sca@ 1002346c     jerror.obj
 0002:00002490       ??_C@_0BG@BALCKDNL@Input?5file?5read?5error@ 10023490     jerror.obj
 0002:000024a8       ??_C@_0CP@IDOBLGGD@Output?5file?5write?5error?5?9?9?9?5out@ 100234a8     jerror.obj
 0002:000024d8       ??_C@_0CI@EKDDDHFF@Fractional?5sampling?5not?5impleme@ 100234d8     jerror.obj
 0002:00002500       ??_C@_0CB@LLDOGNPJ@Huffman?5code?5size?5table?5overflo@ 10023500     jerror.obj
 0002:00002524       ??_C@_0CB@LFBMFPHI@Missing?5Huffman?5code?5table?5entr@ 10023524     jerror.obj
 0002:00002548       ??_C@_0CP@EKFPGPNP@Maximum?5supported?5image?5dimensi@ 10023548     jerror.obj
 0002:00002578       ??_C@_0BB@JJAIKFBB@Empty?5input?5file@ 10023578     jerror.obj
 0002:0000258c       ??_C@_0BM@KEKMMNGA@Premature?5end?5of?5input?5file@ 1002358c     jerror.obj
 0002:000025a8       ??_C@_0DO@OPNPKGO@Cannot?5transcode?5due?5to?5multipl@ 100235a8     jerror.obj
 0002:000025e8       ??_C@_0CH@NIBDNILP@Scan?5script?5does?5not?5transmit?5a@ 100235e8     jerror.obj
 0002:00002610       ??_C@_0CH@EFBBPPCK@Invalid?5color?5quantization?5mode@ 10023610     jerror.obj
 0002:00002638       ??_C@_0BE@EOAAHHJ@Not?5implemented?5yet@ 10023638     jerror.obj
 0002:0000264c       ??_C@_0CO@BEHINNOI@Requested?5feature?5was?5omitted?5a@ 1002364c     jerror.obj
 0002:0000267c       ??_C@_0BM@HJHFKLAF@Backing?5store?5not?5supported@ 1002367c     jerror.obj
 0002:00002698       ??_C@_0CF@BKANFCCL@Huffman?5table?50x?$CF02x?5was?5not?5de@ 10023698     jerror.obj
 0002:000026c0       ??_C@_0CC@BKPLBDLJ@JPEG?5datastream?5contains?5no?5ima@ 100236c0     jerror.obj
 0002:000026e4       ??_C@_0CK@CCHKIENB@Quantization?5table?50x?$CF02x?5was?5n@ 100236e4     jerror.obj
 0002:00002710       ??_C@_0CL@GNLFDFCL@Not?5a?5JPEG?5file?3?5starts?5with?50x@ 10023710     jerror.obj
 0002:0000273c       ??_C@_0BO@DJPLELIB@Insufficient?5memory?5?$CIcase?5?$CFd?$CJ@ 1002373c     jerror.obj
 0002:0000275c       ??_C@_0CO@HPDBAEEA@Cannot?5quantize?5more?5than?5?$CFd?5co@ 1002375c     jerror.obj
 0002:0000278c       ??_C@_0CI@PLMPLCNO@Cannot?5quantize?5to?5fewer?5than?5?$CF@ 1002378c     jerror.obj
 0002:000027b4       ??_C@_0CH@NHMNHHIB@Cannot?5quantize?5to?5more?5than?5?$CFd@ 100237b4     jerror.obj
 0002:000027dc       ??_C@_0CN@IHJJJAFJ@Invalid?5JPEG?5file?5structure?3?5tw@ 100237dc     jerror.obj
 0002:0000280c       ??_C@_0DA@GJIJGINK@Invalid?5JPEG?5file?5structure?3?5mi@ 1002380c     jerror.obj
 0002:0000283c       ??_C@_0CK@HMKECJK@Unsupported?5JPEG?5process?3?5SOF?5t@ 1002383c     jerror.obj
 0002:00002868       ??_C@_0CN@HGJCMLNE@Invalid?5JPEG?5file?5structure?3?5tw@ 10023868     jerror.obj
 0002:00002898       ??_C@_0CM@HONLBDPH@Invalid?5JPEG?5file?5structure?3?5SO@ 10023898     jerror.obj
 0002:000028c4       ??_C@_0CD@POKNOPOF@Failed?5to?5create?5temporary?5file@ 100238c4     jerror.obj
 0002:000028e8       ??_C@_0BO@EEPJGHHI@Read?5failed?5on?5temporary?5file@ 100238e8     jerror.obj
 0002:00002908       ??_C@_0BO@GOBJOAAI@Seek?5failed?5on?5temporary?5file@ 10023908     jerror.obj
 0002:00002928       ??_C@_0DG@KALDLIJB@Write?5failed?5on?5temporary?5file?5@ 10023928     jerror.obj
 0002:00002960       ??_C@_0CK@EPADOAKC@Application?5transferred?5too?5few@ 10023960     jerror.obj
 0002:0000298c       ??_C@_0BP@BPKOBOIP@Unsupported?5marker?5type?50x?$CF02x@ 1002398c     jerror.obj
 0002:000029ac       ??_C@_0CD@GCLFJCHC@Virtual?5array?5controller?5messed@ 100239ac     jerror.obj
 0002:000029d0       ??_C@_0CH@LJLHCCHC@Image?5too?5wide?5for?5this?5impleme@ 100239d0     jerror.obj
 0002:000029f8       ??_C@_0BF@EKLGFGNM@Read?5from?5XMS?5failed@ 100239f8     jerror.obj
 0002:00002a10       ??_C@_0BE@FDPDCBIN@Write?5to?5XMS?5failed@ 10023a10     jerror.obj
 0002:00002a24       ??_C@_0CD@IMBKIDCD@Copyright?5?$CIC?$CJ?51998?0?5Thomas?5G?4?5L@ 10023a24     jerror.obj
 0002:00002a48       ??_C@_0BA@LIJBPGPA@6b?5?527?9Mar?91998@ 10023a48     jerror.obj
 0002:00002a58       ??_C@_0DO@EGLODMBB@Caution?3?5quantization?5tables?5ar@ 10023a58     jerror.obj
 0002:00002a98       ??_C@_0EC@EHPKAOHA@Adobe?5APP14?5marker?3?5version?5?$CFd?0@ 10023a98     jerror.obj
 0002:00002adc       ??_C@_0CK@HCPFFNKJ@Unknown?5APP0?5marker?5?$CInot?5JFIF?$CJ?0@ 10023adc     jerror.obj
 0002:00002b08       ??_C@_0CM@CAEPHFAA@Unknown?5APP14?5marker?5?$CInot?5Adobe@ 10023b08     jerror.obj
 0002:00002b34       ??_C@_0CH@KIJGKPAA@Define?5Arithmetic?5Table?50x?$CF02x?3@ 10023b34     jerror.obj
 0002:00002b5c       ??_C@_0BM@MDIEILCE@Define?5Huffman?5Table?50x?$CF02x@ 10023b5c     jerror.obj
 0002:00002b78       ??_C@_0CL@KLDOJIKN@Define?5Quantization?5Table?5?$CFd?5?5p@ 10023b78     jerror.obj
 0002:00002ba4       ??_C@_0BL@EMFIKBEK@Define?5Restart?5Interval?5?$CFu@ 10023ba4     jerror.obj
 0002:00002bc0       ??_C@_0BE@IPCOOGDJ@Freed?5EMS?5handle?5?$CFu@ 10023bc0     jerror.obj
 0002:00002bd4       ??_C@_0BH@GIPOLIGC@Obtained?5EMS?5handle?5?$CFu@ 10023bd4     jerror.obj
 0002:00002bec       ??_C@_0N@HJHFKELG@End?5Of?5Image@ 10023bec     jerror.obj
 0002:00002bfc       ??_C@_0CI@FKGPAJC@?5?5?5?5?5?5?5?5?$CF3d?5?$CF3d?5?$CF3d?5?$CF3d?5?$CF3d?5?$CF3d@ 10023bfc     jerror.obj
 0002:00002c24       ??_C@_0DF@LOKNABIG@JFIF?5APP0?5marker?3?5version?5?$CFd?4?$CF0@ 10023c24     jerror.obj
 0002:00002c5c       ??_C@_0DM@JLHNPIBE@Warning?3?5thumbnail?5image?5size?5d@ 10023c5c     jerror.obj
 0002:00002c98       ??_C@_0CO@KKPHGHBA@JFIF?5extension?5marker?3?5type?50x?$CF@ 10023c98     jerror.obj
 0002:00002cc8       ??_C@_0CB@BADBMAAB@?5?5?5?5with?5?$CFd?5x?5?$CFd?5thumbnail?5imag@ 10023cc8     jerror.obj
 0002:00002cec       ??_C@_0CH@EHHJCMGA@Miscellaneous?5marker?50x?$CF02x?0?5le@ 10023cec     jerror.obj
 0002:00002d14       ??_C@_0BJ@COPODLDN@Unexpected?5marker?50x?$CF02x@ 10023d14     jerror.obj
 0002:00002d30       ??_C@_0CI@GHPOCOCL@?5?5?5?5?5?5?5?5?$CF4u?5?$CF4u?5?$CF4u?5?$CF4u?5?$CF4u?5?$CF4u@ 10023d30     jerror.obj
 0002:00002d58       ??_C@_0CD@CNNAOOFA@Quantizing?5to?5?$CFd?5?$DN?5?$CFd?$CK?$CFd?$CK?$CFd?5col@ 10023d58     jerror.obj
 0002:00002d7c       ??_C@_0BI@NEIBNACE@Quantizing?5to?5?$CFd?5colors@ 10023d7c     jerror.obj
 0002:00002d94       ??_C@_0CE@FDPBEAOO@Selected?5?$CFd?5colors?5for?5quantiza@ 10023d94     jerror.obj
 0002:00002db8       ??_C@_0CF@NIMOLBCP@At?5marker?50x?$CF02x?0?5recovery?5acti@ 10023db8     jerror.obj
 0002:00002de0       ??_C@_05LLAPAOG@RST?$CFd@  10023de0     jerror.obj
 0002:00002de8       ??_C@_0DJ@PCBCLFML@Smoothing?5not?5supported?5with?5no@ 10023de8     jerror.obj
 0002:00002e24       ??_C@_0DK@DMINKOGN@Start?5Of?5Frame?50x?$CF02x?3?5width?$DN?$CFu@ 10023e24     jerror.obj
 0002:00002e60       ??_C@_0BP@EDCAMHHE@?5?5?5?5Component?5?$CFd?3?5?$CFdhx?$CFdv?5q?$DN?$CFd@ 10023e60     jerror.obj
 0002:00002e80       ??_C@_0P@JLCHJELA@Start?5of?5Image@ 10023e80     jerror.obj
 0002:00002e90       ??_C@_0BN@BLOOHNC@Start?5Of?5Scan?3?5?$CFd?5components@ 10023e90     jerror.obj
 0002:00002eb0       ??_C@_0BO@CDEKFGLC@?5?5?5?5Component?5?$CFd?3?5dc?$DN?$CFd?5ac?$DN?$CFd@ 10023eb0     jerror.obj
 0002:00002ed0       ??_C@_0BN@GAMIJLDC@?5?5Ss?$DN?$CFd?0?5Se?$DN?$CFd?0?5Ah?$DN?$CFd?0?5Al?$DN?$CFd@ 10023ed0     jerror.obj
 0002:00002ef0       ??_C@_0BJ@KDCGAOJB@Closed?5temporary?5file?5?$CFs@ 10023ef0     jerror.obj
 0002:00002f0c       ??_C@_0BJ@GOCABEP@Opened?5temporary?5file?5?$CFs@ 10023f0c     jerror.obj
 0002:00002f28       ??_C@_0EC@ELDEPOJP@JFIF?5extension?5marker?3?5JPEG?9com@ 10023f28     jerror.obj
 0002:00002f6c       ??_C@_0DK@JGAPDCJL@JFIF?5extension?5marker?3?5palette?5@ 10023f6c     jerror.obj
 0002:00002fa8       ??_C@_0DG@FCFDGNHE@JFIF?5extension?5marker?3?5RGB?5thum@ 10023fa8     jerror.obj
 0002:00002fe0       ??_C@_0DE@EEJCDLOO@Unrecognized?5component?5IDs?5?$CFd?5?$CF@ 10023fe0     jerror.obj
 0002:00003014       ??_C@_0BE@FOGGKKAO@Freed?5XMS?5handle?5?$CFu@ 10024014     jerror.obj
 0002:00003028       ??_C@_0BH@LJLGPEFF@Obtained?5XMS?5handle?5?$CFu@ 10024028     jerror.obj
 0002:00003040       ??_C@_0CG@KEGHCDOM@Unknown?5Adobe?5color?5transform?5c@ 10024040     jerror.obj
 0002:00003068       ??_C@_0EC@CBCJOINE@Inconsistent?5progression?5sequen@ 10024068     jerror.obj
 0002:000030ac       ??_C@_0DM@PCOGCKJB@Corrupt?5JPEG?5data?3?5?$CFu?5extraneou@ 100240ac     jerror.obj
 0002:000030e8       ??_C@_0DB@PGMEPGHN@Corrupt?5JPEG?5data?3?5premature?5en@ 100240e8     jerror.obj
 0002:0000311c       ??_C@_0CE@PBLDOPKB@Corrupt?5JPEG?5data?3?5bad?5Huffman?5@ 1002411c     jerror.obj
 0002:00003140       ??_C@_0CO@ODCCEDLN@Warning?3?5unknown?5JFIF?5revision?5@ 10024140     jerror.obj
 0002:00003170       ??_C@_0BL@DPFPFMLM@Premature?5end?5of?5JPEG?5file@ 10024170     jerror.obj
 0002:0000318c       ??_C@_0DI@NFMBADOH@Corrupt?5JPEG?5data?3?5found?5marker@ 1002418c     jerror.obj
 0002:000031c4       ??_C@_0CL@BAKCGOKJ@Invalid?5SOS?5parameters?5for?5sequ@ 100241c4     jerror.obj
 0002:000031f0       ??_C@_0CL@OCGBAKPF@Application?5transferred?5too?5man@ 100241f0     jerror.obj
 0002:0000321c       ??_C@_03OFAPEBGM@?$CFs?6@  1002421c     jerror.obj
 0002:00003220       __real@3f8a8bd4            10024220     jidctflt.obj
 0002:00003224       __real@3fb504f3            10024224     jidctflt.obj
 0002:00003228       __real@3fec835e            10024228     jidctflt.obj
 0002:0000322c       __real@40273d75            1002422c     jidctflt.obj
 0002:00003240       ??_C@_07OOOLPGAB@JPEGMEM@  10024240     jmemmgr.obj
 0002:00003248       ??_C@_04BMELEEFH@?$CFu?$CFc@ 10024248     jmemmgr.obj
 0002:00003360       _jZAGTable                 10024360     jutils.obj
 0002:000034a0       _png_sRGB_table            100244a0     png.obj
 0002:000036a0       _png_sRGB_base             100246a0     png.obj
 0002:00003aa0       _png_sRGB_delta            10024aa0     png.obj
 0002:00003cd8       ??_C@_0CB@IKHEGJHB@Too?5many?5bytes?5for?5PNG?5signatur@ 10024cd8     png.obj
 0002:00003cfc       ??_C@_0CD@PGGPKBFM@Potential?5overflow?5in?5png_zallo@ 10024cfc     png.obj
 0002:00003d20       ??_C@_06IMMIJCHC@1?46?447@ 10024d20     png.obj
 0002:00003d28       ??_C@_0BP@LLMNPADO@Application?5built?5with?5libpng?9@ 10024d28     png.obj
 0002:00003d48       ??_C@_0BD@IECHPOPJ@?5but?5running?5with?5@ 10024d48     png.obj
 0002:00003d5c       ??_C@_0BM@FGHKPJNF@Ignoring?5invalid?5time?5value@ 10024d5c     png.obj
 0002:00003d78       ??_C@_0BM@FGGHCFBF@unexpected?5zlib?5return?5code@ 10024d78     png.obj
 0002:00003d94       ??_C@_0BM@DCGHBGGB@unexpected?5end?5of?5LZ?5stream@ 10024d94     png.obj
 0002:00003db0       ??_C@_0BG@MPHEFODE@missing?5LZ?5dictionary@ 10024db0     png.obj
 0002:00003dc8       ??_C@_0O@HJOFHIEK@zlib?5IO?5error@ 10024dc8     png.obj
 0002:00003dd8       ??_C@_0BH@MLOBAKCG@bad?5parameters?5to?5zlib@ 10024dd8     png.obj
 0002:00003df0       ??_C@_0BC@NNBNLNOK@damaged?5LZ?5stream@ 10024df0     png.obj
 0002:00003e04       ??_C@_0BE@OGGJBMCE@insufficient?5memory@ 10024e04     png.obj
 0002:00003e18       ??_C@_09IDFJECNO@truncated@ 10024e18     png.obj
 0002:00003e24       ??_C@_0BJ@EHGGFMEH@unsupported?5zlib?5version@ 10024e24     png.obj
 0002:00003e40       ??_C@_0BH@MPOINNNJ@unexpected?5zlib?5return@ 10024e40     png.obj
 0002:00003e58       ??_C@_0CK@DCDMPLDM@internal?5error?5handling?5cHRM?5co@ 10024e58     png.obj
 0002:00003e84       ??_C@_0BM@CEAELHL@Image?5width?5is?5zero?5in?5IHDR@ 10024e84     png.obj
 0002:00003ea0       ??_C@_0BM@KHHGCJLE@Invalid?5image?5width?5in?5IHDR@ 10024ea0     png.obj
 0002:00003ebc       ??_C@_0CP@HOJKPAHE@Image?5width?5is?5too?5large?5for?5th@ 10024ebc     png.obj
 0002:00003eec       ??_C@_0CH@COHNFPDF@Image?5width?5exceeds?5user?5limit?5@ 10024eec     png.obj
 0002:00003f14       ??_C@_0BN@CMEOFBLN@Image?5height?5is?5zero?5in?5IHDR@ 10024f14     png.obj
 0002:00003f34       ??_C@_0BN@NOEKCPOM@Invalid?5image?5height?5in?5IHDR@ 10024f34     png.obj
 0002:00003f54       ??_C@_0CI@HDNDADNB@Image?5height?5exceeds?5user?5limit@ 10024f54     png.obj
 0002:00003f7c       ??_C@_0BK@OAKOLNFJ@Invalid?5bit?5depth?5in?5IHDR@ 10024f7c     png.obj
 0002:00003f98       ??_C@_0BL@KPIFPGMP@Invalid?5color?5type?5in?5IHDR@ 10024f98     png.obj
 0002:00003fb4       ??_C@_0DB@FGMBGHOJ@Invalid?5color?5type?1bit?5depth?5co@ 10024fb4     png.obj
 0002:00003fe8       ??_C@_0CB@EMHJMLOA@Unknown?5interlace?5method?5in?5IHD@ 10024fe8     png.obj
 0002:0000400c       ??_C@_0CD@DDOOCEDP@Unknown?5compression?5method?5in?5I@ 1002500c     png.obj
 0002:00004030       ??_C@_0DB@CJBLKABO@MNG?5features?5are?5not?5allowed?5in@ 10025030     png.obj
 0002:00004064       ??_C@_0BO@KOOEGEDO@Unknown?5filter?5method?5in?5IHDR@ 10025064     png.obj
 0002:00004084       ??_C@_0BO@PAJOKPHG@Invalid?5filter?5method?5in?5IHDR@ 10025084     png.obj
 0002:000040a4       ??_C@_0BC@MEPNMCAI@Invalid?5IHDR?5data@ 100250a4     png.obj
 0002:000040b8       ??_C@_0BK@FEDMIILC@gamma?5table?5being?5rebuilt@ 100250b8     png.obj
 0002:000040d8       __real@0000000000000000    100250d8     png.obj
 0002:000040e0       __real@3ee4f8b588e368f1    100250e0     png.obj
 0002:000040e8       __real@3fe0000000000000    100250e8     png.obj
 0002:000040f0       __real@406fe00000000000    100250f0     png.obj
 0002:000040f8       __real@40efffe000000000    100250f8     png.obj
 0002:00004100       __real@40f86a0000000000    10025100     png.obj
 0002:00004108       __real@41dfffffffc00000    10025108     png.obj
 0002:00004110       __real@4202a05f20000000    10025110     png.obj
 0002:00004118       __real@430c6bf526340000    10025118     png.obj
 0002:00004120       __real@c1e0000000000000    10025120     png.obj
 0002:00004130       __xmm@41f00000000000000000000000000000 10025130     png.obj
 0002:00004170       ??_C@_0BJ@BIPJEANG@fixed?5point?5overflow?5in?5@ 10025170     pngerror.obj
 0002:0000418c       ??_C@_0BP@OGHIMAJC@Libpng?5jmp_buf?5still?5allocated@ 1002518c     pngerror.obj
 0002:000041ac       ??_C@_0CB@MNPMICGC@Application?5jmp_buf?5size?5change@ 100251ac     pngerror.obj
 0002:000041d0       ??_C@_09MLGAJAED@undefined@ 100251d0     pngerror.obj
 0002:000041dc       ??_C@_0BB@FHIOKKKG@libpng?5error?3?5?$CFs@ 100251dc     pngerror.obj
 0002:000041f0       ??_C@_01EEMJAFIK@?6@       100251f0     pngerror.obj
 0002:000041f4       ??_C@_0BD@OLJIBHNB@libpng?5warning?3?5?$CFs@ 100251f4     pngerror.obj
 0002:00004208       __real@00000000            10025208     pngget.obj
 0002:0000420c       ??_C@_0BM@JALLIJNF@internal?5error?3?5array?5alloc@ 1002520c     pngmem.obj
 0002:00004228       ??_C@_0BO@KBIBCEFP@internal?5error?3?5array?5realloc@ 10025228     pngmem.obj
 0002:00004248       ??_C@_0O@NALGGDJF@Out?5of?5memory@ 10025248     pngmem.obj
 0002:00004278       ??_C@_0P@KIMIGLKH@Not?5a?5PNG?5file@ 10025278     pngpread.obj
 0002:00004288       ??_C@_0CH@NMANOLCN@PNG?5file?5corrupted?5by?5ASCII?5con@ 10025288     pngpread.obj
 0002:000042b0       ??_C@_0BJ@FFGICIDJ@Missing?5IHDR?5before?5IDAT@ 100252b0     pngpread.obj
 0002:000042cc       ??_C@_0BJ@LAKDHAPN@Missing?5PLTE?5before?5IDAT@ 100252cc     pngpread.obj
 0002:000042e8       ??_C@_0BF@DJLIMHLL@Too?5many?5IDATs?5found@ 100252e8     pngpread.obj
 0002:00004300       ??_C@_0BK@CONOMAKG@bad?5adaptive?5filter?5value@ 10025300     pngpread.obj
 0002:00004360       ??_C@_0DK@FFGAMEAC@png_read_update_info?1png_start_@ 10025360     pngread.obj
 0002:0000439c       ??_C@_0DK@INFAHCPB@png_start_read_image?1png_read_u@ 1002539c     pngread.obj
 0002:000043d8       ??_C@_0CB@KCPNIGFM@Invalid?5attempt?5to?5read?5row?5dat@ 100253d8     pngread.obj
 0002:000043fc       ??_C@_0BI@DKBHKBPF@sequential?5row?5overflow@ 100253fc     pngread.obj
 0002:00004414       ??_C@_0CP@OINAJLHB@internal?5sequential?5row?5size?5ca@ 10025414     pngread.obj
 0002:00004448       ??_C@_0EB@BJILBCPL@Interlace?5handling?5should?5be?5tu@ 10025448     pngread.obj
 0002:0000448c       ??_C@_0CJ@NMAOGEBP@Read?5palette?5index?5exceeding?5nu@ 1002548c     pngread.obj
 0002:000044b8       ??_C@_0BG@JDLIFNJD@?4Too?5many?5IDATs?5found@ 100254b8     pngread.obj
 0002:000044d0       ??_C@_0BH@KGKHPFPD@?4?4Too?5many?5IDATs?5found@ 100254d0     pngread.obj
 0002:000044e8       ??_C@_0BL@GPADEDKN@Call?5to?5NULL?5read?5function@ 100254e8     pngrio.obj
 0002:00004504       ??_C@_0L@BAFDDAPG@Read?5Error@ 10025504     pngrio.obj
 0002:00004510       ??_C@_0DL@CAJMFGIG@invalid?5after?5png_start_read_im@ 10025510     pngrtran.obj
 0002:0000454c       ??_C@_0CM@GNKBMBFP@invalid?5before?5the?5PNG?5header?5h@ 1002554c     pngrtran.obj
 0002:00004578       ??_C@_0M@FBBKEIKG@gamma?5value@ 10025578     pngrtran.obj
 0002:00004584       ??_C@_0BN@MDCNHGNN@gamma?5out?5of?5supported?5range@ 10025584     pngrtran.obj
 0002:000045a4       ??_C@_0CE@IFPDIMOB@invalid?5file?5gamma?5in?5png_set_g@ 100255a4     pngrtran.obj
 0002:000045c8       ??_C@_0CG@NENGEGMG@invalid?5screen?5gamma?5in?5png_set@ 100255c8     pngrtran.obj
 0002:000045f0       ??_C@_0DF@DLPECGFI@libpng?5does?5not?5support?5gamma?$CLb@ 100255f0     pngrtran.obj
 0002:00004628       ??_C@_0BO@ENKNLJK@invalid?5background?5gamma?5type@ 10025628     pngrtran.obj
 0002:00004648       ??_C@_0CB@BPJJBEIH@Palette?5is?5NULL?5in?5indexed?5imag@ 10025648     pngrtran.obj
 0002:0000466c       ??_C@_0CF@NLNFFJAO@png_do_encode_alpha?3?5unexpected@ 1002566c     pngrtran.obj
 0002:00004694       ??_C@_0BA@DBGPKIA@NULL?5row?5buffer@ 10025694     pngrtran.obj
 0002:000046a4       ??_C@_0BC@ICIDCBAI@Uninitialized?5row@ 100256a4     pngrtran.obj
 0002:000046b8       ??_C@_0CH@DAMIMNHG@png_do_rgb_to_gray?5found?5nongra@ 100256b8     pngrtran.obj
 0002:000046e0       ??_C@_0CE@PFPGIBHI@png_do_quantize?5returned?5rowbyt@ 100256e0     pngrtran.obj
 0002:00004708       __real@4060000000000000    10025708     pngrtran.obj
 0002:00004710       __real@c1dfffffffc00000    10025710     pngrtran.obj
 0002:000048f0       ??_C@_0CC@CLHKAOCN@PNG?5unsigned?5integer?5out?5of?5ran@ 100258f0     pngrutil.obj
 0002:00004914       ??_C@_0BM@NOACEJPI@bad?5header?5?$CIinvalid?5length?$CJ@ 10025914     pngrutil.obj
 0002:00004930       ??_C@_0BK@EECCAJL@bad?5header?5?$CIinvalid?5type?$CJ@ 10025930     pngrutil.obj
 0002:0000494c       ??_C@_09BJGMGMHA@CRC?5error@ 1002594c     pngrutil.obj
 0002:00004958       ??_C@_0P@KJIHHBLD@?5using?5zstream@ 10025958     pngrutil.obj
 0002:00004968       ??_C@_0BN@KJIAGOEF@invalid?5window?5size?5?$CIlibpng?$CJ@ 10025968     pngrutil.obj
 0002:00004988       ??_C@_09KHIKJOBP@duplicate@ 10025988     pngrutil.obj
 0002:00004994       ??_C@_0N@LIMFFBPG@out?5of?5place@ 10025994     pngrutil.obj
 0002:000049a4       ??_C@_0BJ@CHOIBJOP@ignored?5in?5grayscale?5PNG@ 100259a4     pngrutil.obj
 0002:000049c0       ??_C@_07MALOAKCI@invalid@  100259c0     pngrutil.obj
 0002:000049c8       ??_C@_0L@DABMCDJH@bad?5length@ 100259c8     pngrutil.obj
 0002:000049d4       ??_C@_0CB@KEIBOKCA@No?5space?5in?5chunk?5cache?5for?5sPL@ 100259d4     pngrutil.obj
 0002:000049f8       ??_C@_0BF@JHCGGFHI@malformed?5sPLT?5chunk@ 100259f8     pngrutil.obj
 0002:00004a10       ??_C@_0BK@FFJLCLGE@sPLT?5chunk?5has?5bad?5length@ 10025a10     pngrutil.obj
 0002:00004a2c       ??_C@_0BE@HJCMKPPM@sPLT?5chunk?5too?5long@ 10025a2c     pngrutil.obj
 0002:00004a40       ??_C@_0CE@MCMAFPMA@sPLT?5chunk?5requires?5too?5much?5me@ 10025a40     pngrutil.obj
 0002:00004a64       ??_C@_0BL@MHLOEJAP@invalid?5with?5alpha?5channel@ 10025a64     pngrutil.obj
 0002:00004a80       ??_C@_0O@BGLHAEFA@invalid?5index@ 10025a80     pngrutil.obj
 0002:00004a90       ??_C@_0BD@JCEBGMHJ@invalid?5gray?5level@ 10025a90     pngrutil.obj
 0002:00004aa4       ??_C@_0O@LIIAELDF@invalid?5color@ 10025aa4     pngrutil.obj
 0002:00004ab4       ??_C@_0BI@LAIHDGGP@invalid?5parameter?5count@ 10025ab4     pngrutil.obj
 0002:00004acc       ??_C@_0BL@OJIHHCAK@unrecognized?5equation?5type@ 10025acc     pngrutil.obj
 0002:00004ae8       ??_C@_0N@FNKMFOEC@invalid?5data@ 10025ae8     pngrutil.obj
 0002:00004af8       ??_C@_0N@HLAECGBB@invalid?5unit@ 10025af8     pngrutil.obj
 0002:00004b08       ??_C@_0BB@CJAEGFPG@bad?5width?5format@ 10025b08     pngrutil.obj
 0002:00004b1c       ??_C@_0BD@PGENKNPL@non?9positive?5width@ 10025b1c     pngrutil.obj
 0002:00004b30       ??_C@_0BC@EEJECMAN@bad?5height?5format@ 10025b30     pngrutil.obj
 0002:00004b44       ??_C@_0BE@DNKCMKFH@non?9positive?5height@ 10025b44     pngrutil.obj
 0002:00004b58       ??_C@_0BI@EMEPIKPK@no?5space?5in?5chunk?5cache@ 10025b58     pngrutil.obj
 0002:00004b70       ??_C@_0CE@OGILCCBP@unknown?5chunk?5exceeds?5memory?5li@ 10025b70     pngrutil.obj
 0002:00004b94       ??_C@_0BE@IFBNEDBM@error?5in?5user?5chunk@ 10025b94     pngrutil.obj
 0002:00004ba8       ??_C@_0BG@IANHEEOB@Saving?5unknown?5chunk?3@ 10025ba8     pngrutil.obj
 0002:00004bc0       ??_C@_0EM@CPAIEDFN@forcing?5save?5of?5an?5unhandled?5ch@ 10025bc0     pngrutil.obj
 0002:00004c0c       ??_C@_0BJ@OGKNBOLG@unhandled?5critical?5chunk@ 10025c0c     pngrutil.obj
 0002:00004c28       ??_C@_0N@POFAPNKG@missing?5IHDR@ 10025c28     pngrutil.obj
 0002:00004c38       ??_C@_09PNOMNDOP@too?5short@ 10025c38     pngrutil.obj
 0002:00004c44       ??_C@_0BM@CMIPFLMD@length?5exceeds?5libpng?5limit@ 10025c44     pngrutil.obj
 0002:00004c60       ??_C@_08JAFCJEPG@too?5long@ 10025c60     pngrutil.obj
 0002:00004c6c       ??_C@_0BJ@DILPAFHB@internal?5row?5logic?5error@ 10025c6c     pngrutil.obj
 0002:00004c88       ??_C@_0CE@DMJCLOFE@internal?5row?5size?5calculation?5e@ 10025c88     pngrutil.obj
 0002:00004cac       ??_C@_0BJ@EGFCIELD@internal?5row?5width?5error@ 10025cac     pngrutil.obj
 0002:00004cc8       ??_C@_0CD@FPHNEGJK@invalid?5user?5transform?5pixel?5de@ 10025cc8     pngrutil.obj
 0002:00004cec       ??_C@_0BG@EIEOOJHA@Not?5enough?5image?5data@ 10025cec     pngrutil.obj
 0002:00004d04       ??_C@_0BG@OKGHHCLP@Extra?5compressed?5data@ 10025d04     pngrutil.obj
 0002:00004d1c       ??_C@_0BE@EFPCKDCF@Too?5much?5image?5data@ 10025d1c     pngrutil.obj
 0002:00004d30       ??_C@_0CN@PNKHKIBI@Row?5has?5too?5many?5bytes?5to?5alloc@ 10025d30     pngrutil.obj
 0002:00004dcc       ??_C@_0CO@CLNKJNCD@Invalid?5palette?5size?0?5hIST?5allo@ 10025dcc     pngset.obj
 0002:00004dfc       ??_C@_0CI@FEJILDIH@Insufficient?5memory?5for?5hIST?5ch@ 10025dfc     pngset.obj
 0002:00004e24       ??_C@_0BL@BGONKFBB@Invalid?5pCAL?5equation?5type@ 10025e24     pngset.obj
 0002:00004e40       ??_C@_0BN@FHGDAAAD@Invalid?5pCAL?5parameter?5count@ 10025e40     pngset.obj
 0002:00004e60       ??_C@_0CC@LPAJHANK@Invalid?5format?5for?5pCAL?5paramet@ 10025e60     pngset.obj
 0002:00004e84       ??_C@_0CF@CKIMKPAH@Insufficient?5memory?5for?5pCAL?5pu@ 10025e84     pngset.obj
 0002:00004eac       ??_C@_0CD@PAPNLFE@Insufficient?5memory?5for?5pCAL?5un@ 10025eac     pngset.obj
 0002:00004ed0       ??_C@_0CE@KNDKKCDF@Insufficient?5memory?5for?5pCAL?5pa@ 10025ed0     pngset.obj
 0002:00004ef4       ??_C@_0CH@CAHFGHFJ@Insufficient?5memory?5for?5pCAL?5pa@ 10025ef4     pngset.obj
 0002:00004f1c       ??_C@_0BC@GANANPIA@Invalid?5sCAL?5unit@ 10025f1c     pngset.obj
 0002:00004f30       ??_C@_0BD@ENHOBHJG@Invalid?5sCAL?5width@ 10025f30     pngset.obj
 0002:00004f44       ??_C@_0BE@OBKOEAI@Invalid?5sCAL?5height@ 10025f44     pngset.obj
 0002:00004f58       ??_C@_0CP@EHHAKMDE@Memory?5allocation?5failed?5while?5@ 10025f58     pngset.obj
 0002:00004f88       ??_C@_0BH@IKBNLCFC@Invalid?5palette?5length@ 10025f88     pngset.obj
 0002:00004fa0       ??_C@_0BA@NCKCMMNF@Invalid?5palette@ 10025fa0     pngset.obj
 0002:00004fb0       ??_C@_0BF@EPLDENLO@too?5many?5text?5chunks@ 10025fb0     pngset.obj
 0002:00004fc8       ??_C@_0CG@KOBFBGAM@text?5compression?5mode?5is?5out?5of@ 10025fc8     pngset.obj
 0002:00004ff0       ??_C@_0BK@FPMAJGNB@text?5chunk?3?5out?5of?5memory@ 10025ff0     pngset.obj
 0002:0000500c       ??_C@_0DC@BAKLMMNF@tRNS?5chunk?5has?5out?9of?9range?5sam@ 1002600c     pngset.obj
 0002:00005040       ??_C@_0BF@IBPPODIO@too?5many?5sPLT?5chunks@ 10026040     pngset.obj
 0002:00005058       ??_C@_0BL@FDLCPBMN@png_set_sPLT?3?5invalid?5sPLT@ 10026058     pngset.obj
 0002:00005074       ??_C@_0BD@FCEBHNK@sPLT?5out?5of?5memory@ 10026074     pngset.obj
 0002:00005088       ??_C@_0DE@GDJFMIAK@png_set_unknown_chunks?5now?5expe@ 10026088     pngset.obj
 0002:000050bc       ??_C@_0CL@HCECGJBJ@invalid?5location?5in?5png_set_unk@ 100260bc     pngset.obj
 0002:000050e8       ??_C@_0BI@DHBNAPDO@too?5many?5unknown?5chunks@ 100260e8     pngset.obj
 0002:00005100       ??_C@_0BN@IMBDGIBC@unknown?5chunk?3?5out?5of?5memory@ 10026100     pngset.obj
 0002:00005420       ??_C@_0CG@FFCAHEBJ@png_set_filler?5not?5supported?5on@ 10026420     pngtrans.obj
 0002:00005448       _baseDitherMatrix          10026448     splashscreen_gfx_impl.obj
 0002:00005578       ??_C@_07HCPCJKKB@?$EA100pct@ 10026578     splashscreen_impl.obj
 0002:00005580       ??_C@_03LEEGEJPE@pct@      10026580     splashscreen_impl.obj
 0002:00005584       ??_C@_01EOFPKCAF@?$EA@     10026584     splashscreen_impl.obj
 0002:00005588       ??_C@_06PFFBCHML@?$CFs?$CFd?$CFs@ 10026588     splashscreen_impl.obj
 0002:00005590       ??_C@_01FJMABOPO@x@        10026590     splashscreen_impl.obj
 0002:00005594       ??_C@_04HDOCAJNK@?$CFs?$CFs@ 10026594     splashscreen_impl.obj
 0002:0000559c       ??_C@_08JBCIEEFM@?$CF?4?$CKs?$CFs?$CFs@ 1002659c     splashscreen_impl.obj
 0002:000055a8       ??_C@_01KDCPPGHE@r@        100265a8     splashscreen_impl.obj
 0002:000055ac       __real@42c80000            100265ac     splashscreen_impl.obj
 0002:000055b0       __real@400199999999999a    100265b0     splashscreen_png.obj
 0002:000055b8       ??_C@_0L@DMJGLJCL@JavaSplash@ 100265b8     splashscreen_sys.obj
 0002:000055c4       __real@42c00000            100265c4     splashscreen_sys.obj
 0002:000055c8       ??_C@_0M@JKPININF@J2D_UISCALE@ 100265c8     systemScale.obj
 0002:000055d4       ??_C@_0L@DMFDIJCG@shcore?4dll@ 100265d4     systemScale.obj
 0002:000055e0       ??_C@_0BB@MAMHPNNC@GetDpiForMonitor@ 100265e0     systemScale.obj
 0002:000055f4       __real@bf800000            100265f4     systemScale.obj
 0002:000055f8       __real@c0000000            100265f8     systemScale.obj
 0002:00005600       __length_code              10026600     trees.obj
 0002:00005700       __dist_code                10026700     trees.obj
 0002:000088f8       _z_errmsg                  100298f8     zutil.obj
 0002:00008920       ??_C@_0BA@MOKMMFOD@need?5dictionary@ 10029920     zutil.obj
 0002:00008930       ??_C@_0L@FNAOCBOG@stream?5end@ 10029930     zutil.obj
 0002:0000893c       ??_C@_0L@KIJFAKBJ@file?5error@ 1002993c     zutil.obj
 0002:00008948       ??_C@_0N@MKKNPMJD@stream?5error@ 10029948     zutil.obj
 0002:00008958       ??_C@_0L@HAHMBNLP@data?5error@ 10029958     zutil.obj
 0002:00008964       ??_C@_0N@DFPGLBGC@buffer?5error@ 10029964     zutil.obj
 0002:00008974       ??_C@_0BF@CJFPCCEG@incompatible?5version@ 10029974     zutil.obj
 0002:00008990       __sz_USER32_dll            10029990     user32:USER32.dll
 0002:0000899c       ??_C@_1BK@DBDEIDLH@?$AAK?$AAE?$AAR?$AAN?$AAE?$AAL?$AA3?$AA2?$AA?4?$AAD?$AAL?$AAL@ 1002999c     delayimp:delayhlp.obj
 0002:000089b8       ??_C@_0BI@OMNLIJDB@AcquireSRWLockExclusive@ 100299b8     delayimp:delayhlp.obj
 0002:000089d0       ??_C@_0BI@HMIEPCNJ@ReleaseSRWLockExclusive@ 100299d0     delayimp:delayhlp.obj
 0002:000089e8       ___pfnDliNotifyHook2       100299e8     delayimp:delayhk2.obj
 0002:000089ec       ___pfnDliFailureHook2      100299ec     delayimp:delayhk1.obj
 0002:00008a40       __pDefaultRawDllMain       10029a40     MSVCRT:dll_dllmain.obj
 0002:00008a40       __pRawDllMain              10029a40     MSVCRT:dll_dllmain.obj
 0002:00008a48       __load_config_used         10029a48     MSVCRT:loadcfg.obj
 0002:00008b80       ___safe_se_handler_table   10029b80     <linker-defined>
 0002:00008b84       ___volatile_metadata       10029b84     <linker-defined>
 0002:00008f58       ___rtc_iaa                 10029f58     MSVCRT:initsect.obj
 0002:00008f5c       ___rtc_izz                 10029f5c     MSVCRT:initsect.obj
 0002:00008f60       ___rtc_taa                 10029f60     MSVCRT:initsect.obj
 0002:00008f64       ___rtc_tzz                 10029f64     MSVCRT:initsect.obj
 0002:00008fec       __DELAY_IMPORT_DESCRIPTOR_user32_dll 10029fec     user32:USER32.dll
 0002:0000900c       __NULL_DELAY_IMPORT_DESCRIPTOR 1002a00c     user32:USER32.dll
 0002:000090ac       \177USER32_NULL_THUNK_DATA_DLN 1002a0ac     user32:USER32.dll
 0002:000092b8       \177USER32_NULL_THUNK_DATA_DLB 1002a2b8     user32:USER32.dll
 0002:0000966c       __IMPORT_DESCRIPTOR_KERNEL32 1002a66c     kernel32:KERNEL32.dll
 0002:00009680       __IMPORT_DESCRIPTOR_GDI32  1002a680     gdi32:GDI32.dll
 0002:00009694       __IMPORT_DESCRIPTOR_java   1002a694     java:java.dll
 0002:000096a8       __IMPORT_DESCRIPTOR_VCRUNTIME140 1002a6a8     vcruntime:VCRUNTIME140.dll
 0002:000096bc       __IMPORT_DESCRIPTOR_api-ms-win-crt-stdio-l1-1-0 1002a6bc     ucrt:api-ms-win-crt-stdio-l1-1-0.dll
 0002:000096d0       __IMPORT_DESCRIPTOR_api-ms-win-crt-heap-l1-1-0 1002a6d0     ucrt:api-ms-win-crt-heap-l1-1-0.dll
 0002:000096e4       __IMPORT_DESCRIPTOR_api-ms-win-crt-string-l1-1-0 1002a6e4     ucrt:api-ms-win-crt-string-l1-1-0.dll
 0002:000096f8       __IMPORT_DESCRIPTOR_api-ms-win-crt-convert-l1-1-0 1002a6f8     ucrt:api-ms-win-crt-convert-l1-1-0.dll
 0002:0000970c       __IMPORT_DESCRIPTOR_api-ms-win-crt-runtime-l1-1-0 1002a70c     ucrt:api-ms-win-crt-runtime-l1-1-0.dll
 0002:00009720       __IMPORT_DESCRIPTOR_api-ms-win-crt-environment-l1-1-0 1002a720     ucrt:api-ms-win-crt-environment-l1-1-0.dll
 0002:00009734       __IMPORT_DESCRIPTOR_api-ms-win-crt-math-l1-1-0 1002a734     ucrt:api-ms-win-crt-math-l1-1-0.dll
 0002:00009748       __NULL_IMPORT_DESCRIPTOR   1002a748     kernel32:KERNEL32.dll
 0003:00000004       ___security_cookie_complement 1002b004     MSVCRT:gs_cookie.obj
 0003:00000008       ___security_cookie         1002b008     MSVCRT:gs_cookie.obj
 0003:0000000c       __fltused                  1002b00c     MSVCRT:fltused.obj
 0003:00000010       ___isa_enabled             1002b010     MSVCRT:cpu_disp.obj
 0003:00000020       ___scrt_native_dllmain_reason 1002b020     MSVCRT:utility.obj
 0003:00000030       ___scrt_ucrt_dll_is_in_use 1002b030     MSVCRT:ucrt_stubs.obj
 0003:00000034       __imp__GetMessageA@16      1002b034     user32:USER32.dll
 0003:00000038       __imp__LoadCursorA@8       1002b038     user32:USER32.dll
 0003:0000003c       __imp__TranslateMessage@4  1002b03c     user32:USER32.dll
 0003:00000040       __imp__DispatchMessageA@4  1002b040     user32:USER32.dll
 0003:00000044       __imp__PostMessageA@16     1002b044     user32:USER32.dll
 0003:00000048       __imp__DefWindowProcA@16   1002b048     user32:USER32.dll
 0003:0000004c       __imp__PostQuitMessage@4   1002b04c     user32:USER32.dll
 0003:00000050       __imp__RegisterClassExA@4  1002b050     user32:USER32.dll
 0003:00000054       __imp__CreateWindowExA@48  1002b054     user32:USER32.dll
 0003:00000058       __imp__DestroyWindow@4     1002b058     user32:USER32.dll
 0003:0000005c       __imp__ShowWindow@8        1002b05c     user32:USER32.dll
 0003:00000060       __imp__UpdateLayeredWindow@36 1002b060     user32:USER32.dll
 0003:00000064       __imp__MoveWindow@24       1002b064     user32:USER32.dll
 0003:00000068       __imp__IsWindowVisible@4   1002b068     user32:USER32.dll
 0003:0000006c       __imp__SetTimer@16         1002b06c     user32:USER32.dll
 0003:00000070       __imp__KillTimer@8         1002b070     user32:USER32.dll
 0003:00000074       __imp__GetSystemMetrics@4  1002b074     user32:USER32.dll
 0003:00000078       __imp__UpdateWindow@4      1002b078     user32:USER32.dll
 0003:0000007c       __imp__GetDC@4             1002b07c     user32:USER32.dll
 0003:00000080       __imp__ReleaseDC@8         1002b080     user32:USER32.dll
 0003:00000084       __imp__BeginPaint@8        1002b084     user32:USER32.dll
 0003:00000088       __imp__EndPaint@8          1002b088     user32:USER32.dll
 0003:0000008c       __imp__SetWindowRgn@12     1002b08c     user32:USER32.dll
 0003:00000090       __imp__InvalidateRect@12   1002b090     user32:USER32.dll
 0003:00000094       __imp__GetWindowRect@8     1002b094     user32:USER32.dll
 0003:00000098       __imp__SetCursorPos@8      1002b098     user32:USER32.dll
 0003:0000009c       __imp__SetCursor@4         1002b09c     user32:USER32.dll
 0003:000000a0       __imp__GetCursorPos@4      1002b0a0     user32:USER32.dll
 0003:000000a4       __imp__WindowFromPoint@8   1002b0a4     user32:USER32.dll
 0003:000000a8       __imp__GetWindowLongA@8    1002b0a8     user32:USER32.dll
 0003:000000ac       __imp__SetWindowLongA@12   1002b0ac     user32:USER32.dll
 0003:000000b0       __imp__MonitorFromPoint@12 1002b0b0     user32:USER32.dll
 0003:000000b4       \177USER32_NULL_THUNK_DATA_DLA 1002b0b4     user32:USER32.dll
 0003:000000c0       _splashIsVisible           1002b0c0     splashscreen_impl.obj
 0003:00002e40       __hmod__USER32_dll         1002de40     user32:USER32.dll
 0003:00002e44       ?DloadKernel32@@3PAUHINSTANCE__@@A 1002de44     delayimp:delayhlp.obj
 0003:00002e48       ?DloadAcquireSRWLockExclusive@@3P6GXPAK@ZA 1002de48     delayimp:delayhlp.obj
 0003:00002e4c       ?DloadReleaseSRWLockExclusive@@3P6GXPAK@ZA 1002de4c     delayimp:delayhlp.obj
 0003:00002e50       ?DloadSrwLock@@3KA         1002de50     delayimp:delayhlp.obj
 0003:00002e54       ?DloadSectionLockCount@@3KA 1002de54     delayimp:delayhlp.obj
 0003:00002e58       ?DloadSectionOldProtection@@3KA 1002de58     delayimp:delayhlp.obj
 0003:00002e5c       ?DloadSectionCommitPermanent@@3KA 1002de5c     delayimp:delayhlp.obj
 0003:00003180       ___isa_available           1002e180     MSVCRT:cpu_disp.obj
 0003:00003184       ___favor                   1002e184     MSVCRT:cpu_disp.obj
 0003:00003188       ?__type_info_root_node@@3U__type_info_node@@A 1002e188     MSVCRT:tncleanup.obj
 0003:00003190       ___scrt_current_native_startup_state 1002e190     MSVCRT:utility.obj
 0003:00003194       ___scrt_native_startup_lock 1002e194     MSVCRT:utility.obj
 0003:000031b4       ___scrt_debugger_hook_flag 1002e1b4     MSVCRT:utility_desktop.obj
 0003:000031b8       ?_OptionsStorage@?1??__local_stdio_scanf_options@@9@9 1002e1b8     <common>
 0003:000031c0       ?_OptionsStorage@?1??__local_stdio_printf_options@@9@9 1002e1c0     <common>
 0003:000031c8       ___dyn_tls_init_callback   1002e1c8     <common>

 entry point at        0001:0001f690

 Static symbols

 0000:fffcf000       .debug$S                   10000000     splashscreen.exp
 0000:fffcf000       .debug$S                   10000000     vcruntime:VCRUNTIME140.dll
 0000:fffcf000       .debug$S                   10000000     vcruntime:VCRUNTIME140.dll
 0000:fffcf000       .debug$S                   10000000     vcruntime:VCRUNTIME140.dll
 0000:fffcf000       .debug$S                   10000000     vcruntime:VCRUNTIME140.dll
 0000:fffcf000       .debug$S                   10000000     vcruntime:VCRUNTIME140.dll
 0000:fffcf000       .debug$S                   10000000     vcruntime:VCRUNTIME140.dll
 0000:fffcf000       .debug$S                   10000000     vcruntime:VCRUNTIME140.dll
 0000:fffcf000       .debug$S                   10000000     vcruntime:VCRUNTIME140.dll
 0000:fffcf000       .debug$S                   10000000     vcruntime:VCRUNTIME140.dll
 0000:fffcf000       .debug$S                   10000000     vcruntime:VCRUNTIME140.dll
 0000:fffcf000       .debug$S                   10000000     vcruntime:VCRUNTIME140.dll
 0000:fffcf000       .debug$S                   10000000     vcruntime:VCRUNTIME140.dll
 0000:fffcf000       .debug$S                   10000000     ucrt:api-ms-win-crt-convert-l1-1-0.dll
 0000:fffcf000       .debug$S                   10000000     ucrt:api-ms-win-crt-convert-l1-1-0.dll
 0000:fffcf000       .debug$S                   10000000     ucrt:api-ms-win-crt-convert-l1-1-0.dll
 0000:fffcf000       .debug$S                   10000000     ucrt:api-ms-win-crt-environment-l1-1-0.dll
 0000:fffcf000       .debug$S                   10000000     ucrt:api-ms-win-crt-heap-l1-1-0.dll
 0000:fffcf000       .debug$S                   10000000     ucrt:api-ms-win-crt-heap-l1-1-0.dll
 0000:fffcf000       .debug$S                   10000000     ucrt:api-ms-win-crt-heap-l1-1-0.dll
 0000:fffcf000       .debug$S                   10000000     ucrt:api-ms-win-crt-heap-l1-1-0.dll
 0000:fffcf000       .debug$S                   10000000     ucrt:api-ms-win-crt-math-l1-1-0.dll
 0000:fffcf000       .debug$S                   10000000     ucrt:api-ms-win-crt-math-l1-1-0.dll
 0000:fffcf000       .debug$S                   10000000     ucrt:api-ms-win-crt-math-l1-1-0.dll
 0000:fffcf000       .debug$S                   10000000     ucrt:api-ms-win-crt-math-l1-1-0.dll
 0000:fffcf000       .debug$S                   10000000     ucrt:api-ms-win-crt-math-l1-1-0.dll
 0000:fffcf000       .debug$S                   10000000     ucrt:api-ms-win-crt-math-l1-1-0.dll
 0000:fffcf000       .debug$S                   10000000     ucrt:api-ms-win-crt-runtime-l1-1-0.dll
 0000:fffcf000       .debug$S                   10000000     ucrt:api-ms-win-crt-runtime-l1-1-0.dll
 0000:fffcf000       .debug$S                   10000000     ucrt:api-ms-win-crt-runtime-l1-1-0.dll
 0000:fffcf000       .debug$S                   10000000     ucrt:api-ms-win-crt-runtime-l1-1-0.dll
 0000:fffcf000       .debug$S                   10000000     ucrt:api-ms-win-crt-runtime-l1-1-0.dll
 0000:fffcf000       .debug$S                   10000000     ucrt:api-ms-win-crt-runtime-l1-1-0.dll
 0000:fffcf000       .debug$S                   10000000     ucrt:api-ms-win-crt-runtime-l1-1-0.dll
 0000:fffcf000       .debug$S                   10000000     ucrt:api-ms-win-crt-runtime-l1-1-0.dll
 0000:fffcf000       .debug$S                   10000000     ucrt:api-ms-win-crt-runtime-l1-1-0.dll
 0000:fffcf000       .debug$S                   10000000     ucrt:api-ms-win-crt-runtime-l1-1-0.dll
 0000:fffcf000       .debug$S                   10000000     ucrt:api-ms-win-crt-runtime-l1-1-0.dll
 0000:fffcf000       .debug$S                   10000000     ucrt:api-ms-win-crt-runtime-l1-1-0.dll
 0000:fffcf000       .debug$S                   10000000     ucrt:api-ms-win-crt-runtime-l1-1-0.dll
 0000:fffcf000       .debug$S                   10000000     ucrt:api-ms-win-crt-runtime-l1-1-0.dll
 0000:fffcf000       .debug$S                   10000000     ucrt:api-ms-win-crt-runtime-l1-1-0.dll
 0000:fffcf000       .debug$S                   10000000     ucrt:api-ms-win-crt-stdio-l1-1-0.dll
 0000:fffcf000       .debug$S                   10000000     ucrt:api-ms-win-crt-stdio-l1-1-0.dll
 0000:fffcf000       .debug$S                   10000000     ucrt:api-ms-win-crt-stdio-l1-1-0.dll
 0000:fffcf000       .debug$S                   10000000     ucrt:api-ms-win-crt-stdio-l1-1-0.dll
 0000:fffcf000       .debug$S                   10000000     ucrt:api-ms-win-crt-stdio-l1-1-0.dll
 0000:fffcf000       .debug$S                   10000000     ucrt:api-ms-win-crt-stdio-l1-1-0.dll
 0000:fffcf000       .debug$S                   10000000     ucrt:api-ms-win-crt-stdio-l1-1-0.dll
 0000:fffcf000       .debug$S                   10000000     ucrt:api-ms-win-crt-stdio-l1-1-0.dll
 0000:fffcf000       .debug$S                   10000000     ucrt:api-ms-win-crt-stdio-l1-1-0.dll
 0000:fffcf000       .debug$S                   10000000     ucrt:api-ms-win-crt-stdio-l1-1-0.dll
 0000:fffcf000       .debug$S                   10000000     ucrt:api-ms-win-crt-stdio-l1-1-0.dll
 0000:fffcf000       .debug$S                   10000000     ucrt:api-ms-win-crt-stdio-l1-1-0.dll
 0000:fffcf000       .debug$S                   10000000     ucrt:api-ms-win-crt-stdio-l1-1-0.dll
 0000:fffcf000       .debug$S                   10000000     ucrt:api-ms-win-crt-stdio-l1-1-0.dll
 0000:fffcf000       .debug$S                   10000000     ucrt:api-ms-win-crt-stdio-l1-1-0.dll
 0000:fffcf000       .debug$S                   10000000     ucrt:api-ms-win-crt-stdio-l1-1-0.dll
 0000:fffcf000       .debug$S                   10000000     ucrt:api-ms-win-crt-string-l1-1-0.dll
 0000:fffcf000       .debug$S                   10000000     ucrt:api-ms-win-crt-string-l1-1-0.dll
 0000:fffcf000       .debug$S                   10000000     ucrt:api-ms-win-crt-string-l1-1-0.dll
 0000:fffcf000       .debug$S                   10000000     ucrt:api-ms-win-crt-string-l1-1-0.dll
 0000:fffcf000       .debug$S                   10000000     ucrt:api-ms-win-crt-utility-l1-1-0.dll
 0002:fffdf000       .idata$6                   10000000     ucrt:api-ms-win-crt-utility-l1-1-0.dll
 0000:fffcf000       .debug$S                   10000000     gdi32:GDI32.dll
 0000:fffcf000       .debug$S                   10000000     gdi32:GDI32.dll
 0000:fffcf000       .debug$S                   10000000     gdi32:GDI32.dll
 0000:fffcf000       .debug$S                   10000000     gdi32:GDI32.dll
 0000:fffcf000       .debug$S                   10000000     gdi32:GDI32.dll
 0000:fffcf000       .debug$S                   10000000     gdi32:GDI32.dll
 0000:fffcf000       .debug$S                   10000000     gdi32:GDI32.dll
 0000:fffcf000       .debug$S                   10000000     gdi32:GDI32.dll
 0000:fffcf000       .debug$S                   10000000     gdi32:GDI32.dll
 0000:fffcf000       .debug$S                   10000000     gdi32:GDI32.dll
 0000:fffcf000       .debug$S                   10000000     gdi32:GDI32.dll
 0000:fffcf000       .debug$S                   10000000     gdi32:GDI32.dll
 0000:fffcf000       .debug$S                   10000000     gdi32:GDI32.dll
 0000:fffcf000       .debug$S                   10000000     kernel32:KERNEL32.dll
 0000:fffcf000       .debug$S                   10000000     kernel32:KERNEL32.dll
 0000:fffcf000       .debug$S                   10000000     kernel32:KERNEL32.dll
 0000:fffcf000       .debug$S                   10000000     kernel32:KERNEL32.dll
 0000:fffcf000       .debug$S                   10000000     kernel32:KERNEL32.dll
 0000:fffcf000       .debug$S                   10000000     kernel32:KERNEL32.dll
 0000:fffcf000       .debug$S                   10000000     kernel32:KERNEL32.dll
 0000:fffcf000       .debug$S                   10000000     kernel32:KERNEL32.dll
 0000:fffcf000       .debug$S                   10000000     kernel32:KERNEL32.dll
 0000:fffcf000       .debug$S                   10000000     kernel32:KERNEL32.dll
 0000:fffcf000       .debug$S                   10000000     kernel32:KERNEL32.dll
 0000:fffcf000       .debug$S                   10000000     kernel32:KERNEL32.dll
 0000:fffcf000       .debug$S                   10000000     kernel32:KERNEL32.dll
 0000:fffcf000       .debug$S                   10000000     kernel32:KERNEL32.dll
 0000:fffcf000       .debug$S                   10000000     kernel32:KERNEL32.dll
 0000:fffcf000       .debug$S                   10000000     kernel32:KERNEL32.dll
 0000:fffcf000       .debug$S                   10000000     kernel32:KERNEL32.dll
 0000:fffcf000       .debug$S                   10000000     kernel32:KERNEL32.dll
 0000:fffcf000       .debug$S                   10000000     kernel32:KERNEL32.dll
 0000:fffcf000       .debug$S                   10000000     kernel32:KERNEL32.dll
 0000:fffcf000       .debug$S                   10000000     kernel32:KERNEL32.dll
 0000:fffcf000       .debug$S                   10000000     kernel32:KERNEL32.dll
 0000:fffcf000       .debug$S                   10000000     kernel32:KERNEL32.dll
 0000:fffcf000       .debug$S                   10000000     kernel32:KERNEL32.dll
 0000:fffcf000       .debug$S                   10000000     kernel32:KERNEL32.dll
 0000:fffcf000       .debug$S                   10000000     kernel32:KERNEL32.dll
 0000:fffcf000       .debug$S                   10000000     kernel32:KERNEL32.dll
 0000:fffcf000       .debug$S                   10000000     kernel32:KERNEL32.dll
 0000:fffcf000       .debug$S                   10000000     kernel32:KERNEL32.dll
 0000:fffcf000       .debug$S                   10000000     user32:USER32.dll
 0000:fffcf000       .debug$S                   10000000     user32:USER32.dll
 0000:fffcf000       .debug$S                   10000000     user32:USER32.dll
 0000:fffcf000       .debug$S                   10000000     user32:USER32.dll
 0000:fffcf000       .debug$S                   10000000     user32:USER32.dll
 0000:fffcf000       .debug$S                   10000000     user32:USER32.dll
 0000:fffcf000       .debug$S                   10000000     user32:USER32.dll
 0000:fffcf000       .debug$S                   10000000     user32:USER32.dll
 0000:fffcf000       .debug$S                   10000000     user32:USER32.dll
 0000:fffcf000       .debug$S                   10000000     user32:USER32.dll
 0000:fffcf000       .debug$S                   10000000     user32:USER32.dll
 0000:fffcf000       .debug$S                   10000000     user32:USER32.dll
 0000:fffcf000       .debug$S                   10000000     user32:USER32.dll
 0000:fffcf000       .debug$S                   10000000     user32:USER32.dll
 0000:fffcf000       .debug$S                   10000000     user32:USER32.dll
 0000:fffcf000       .debug$S                   10000000     user32:USER32.dll
 0000:fffcf000       .debug$S                   10000000     user32:USER32.dll
 0000:fffcf000       .debug$S                   10000000     user32:USER32.dll
 0000:fffcf000       .debug$S                   10000000     user32:USER32.dll
 0000:fffcf000       .debug$S                   10000000     user32:USER32.dll
 0000:fffcf000       .debug$S                   10000000     user32:USER32.dll
 0000:fffcf000       .debug$S                   10000000     user32:USER32.dll
 0000:fffcf000       .debug$S                   10000000     user32:USER32.dll
 0000:fffcf000       .debug$S                   10000000     user32:USER32.dll
 0000:fffcf000       .debug$S                   10000000     user32:USER32.dll
 0000:fffcf000       .debug$S                   10000000     user32:USER32.dll
 0000:fffcf000       .debug$S                   10000000     user32:USER32.dll
 0000:fffcf000       .debug$S                   10000000     user32:USER32.dll
 0000:fffcf000       .debug$S                   10000000     user32:USER32.dll
 0000:fffcf000       .debug$S                   10000000     user32:USER32.dll
 0000:fffcf000       .debug$S                   10000000     user32:USER32.dll
 0000:fffcf000       .debug$S                   10000000     user32:USER32.dll
 0000:fffcf000       .debug$S                   10000000     java:java.dll
 0001:00000000       _deflate_stored            10001000 f   deflate.obj
 0001:0000037e       _deflate_fast              1000137e f   deflate.obj
 0001:000006bc       _deflate_slow              100016bc f   deflate.obj
 0001:00000af6       _fill_window               10001af6 f   deflate.obj
 0001:00000c8d       _flush_pending             10001c8d f   deflate.obj
 0001:00000cd6       _longest_match             10001cd6 f   deflate.obj
 0001:00000e40       _read_buf                  10001e40 f   deflate.obj
 0001:00000eaa       _slide_hash                10001eaa f   deflate.obj
 0001:00000f17       _DGifBufferedInput         10001f17 f   dgif_lib.obj
 0001:00001053       _DGifDecompressInput       10002053 f   dgif_lib.obj
 0001:000010f0       _DGifDecompressLine        100020f0 f   dgif_lib.obj
 0001:000016d7       _DGifGetPrefixChar         100026d7 f   dgif_lib.obj
 0001:000018b8       _DGifGetWord               100028b8 f   dgif_lib.obj
 0001:00001a42       _DGifSetupDecompress       10002a42 f   dgif_lib.obj
 0001:00001c70       _InternalRead              10002c70 f   dgif_lib.obj
 0001:0000372d       $LN761                     1000472d     inflate.obj
 0001:000039ab       _inflateStateCheck         100049ab f   inflate.obj
 0001:000039de       _updatewindow              100049de f   inflate.obj
 0001:0000424f       _default_decompress_parms  1000524f f   jdapimin.obj
 0001:00004445       $LN18                      10005445     jdapimin.obj
 0001:00004459       $LN17                      10005459     jdapimin.obj
 0001:00004794       _output_pass_setup         10005794 f   jdapistd.obj
 0001:00004839       _consume_data              10005839 f   jdcoefct.obj
 0001:00004a2e       _decompress_data           10005a2e f   jdcoefct.obj
 0001:00004baa       _decompress_onepass        10005baa f   jdcoefct.obj
 0001:00004e06       _decompress_smooth_data    10005e06 f   jdcoefct.obj
 0001:000053f2       _dummy_consume_data        100063f2 f   jdcoefct.obj
 0001:000054f4       _smoothing_ok              100064f4 f   jdcoefct.obj
 0001:0000561d       _start_iMCU_row            1000661d f   jdcoefct.obj
 0001:0000565d       _start_input_pass          1000665d f   jdcoefct.obj
 0001:00005670       _start_output_pass         10006670 f   jdcoefct.obj
 0001:000056ad       _build_ycc_rgb_table       100066ad f   jdcolor.obj
 0001:00005766       _gray_rgb_convert          10006766 f   jdcolor.obj
 0001:000057c9       _grayscale_convert         100067c9 f   jdcolor.obj
 0001:00005953       _null_convert              10006953 f   jdcolor.obj
 0001:000059d8       _start_pass_dcolor         100069d8 f   jdcolor.obj
 0001:000059d8       _finish_pass_1_quant       100069d8 f   jquant1.obj
 0001:000059d8       _finish_pass2              100069d8 f   jquant2.obj
 0001:000059d8       _closeMem                  100069d8 f   splashscreen_impl.obj
 0001:000059d8       _stream_term_source        100069d8 f   splashscreen_jpeg.obj
 0001:000059db       _ycc_rgb_convert           100069db f   jdcolor.obj
 0001:00005b15       _ycck_cmyk_convert         10006b15 f   jdcolor.obj
 0001:00005cdb       _start_pass                10006cdb f   jddctmgr.obj
 0001:00005eb1       _decode_mcu                10006eb1 f   jdhuff.obj
 0001:0000674b       _process_restart           1000774b f   jdhuff.obj
 0001:000067b7       _start_pass_huff_decoder   100077b7 f   jdhuff.obj
 0001:000068dd       _consume_markers           100078dd f   jdinput.obj
 0001:00006982       _finish_input_pass         10007982 f   jdinput.obj
 0001:00006993       _initial_setup             10007993 f   jdinput.obj
 0001:00006b9f       _latch_quant_tables        10007b9f f   jdinput.obj
 0001:00006c2f       _per_scan_setup            10007c2f f   jdinput.obj
 0001:00006da6       _reset_input_controller    10007da6 f   jdinput.obj
 0001:00006de0       _start_input_pass          10007de0 f   jdinput.obj
 0001:00006e19       _alloc_funny_pointers      10007e19 f   jdmainct.obj
 0001:00006f8b       _make_funny_pointers       10007f8b f   jdmainct.obj
 0001:000070c4       _process_data_context_main 100080c4 f   jdmainct.obj
 0001:000071e5       _process_data_crank_post   100081e5 f   jdmainct.obj
 0001:00007208       _process_data_simple_main  10008208 f   jdmainct.obj
 0001:00007271       _set_bottom_pointers       10008271 f   jdmainct.obj
 0001:00007309       _set_wraparound_pointers   10008309 f   jdmainct.obj
 0001:000073e4       _start_pass_main           100083e4 f   jdmainct.obj
 0001:0000744e       _examine_app0              1000844e f   jdmarker.obj
 0001:0000767d       _examine_app14             1000867d f   jdmarker.obj
 0001:00007749       _first_marker              10008749 f   jdmarker.obj
 0001:000077d9       _get_dht                   100087d9 f   jdmarker.obj
 0001:00007ac0       _get_dqt                   10008ac0 f   jdmarker.obj
 0001:00007d37       _get_dri                   10008d37 f   jdmarker.obj
 0001:00007e2d       _get_interesting_appn      10008e2d f   jdmarker.obj
 0001:00007f78       _get_sof                   10008f78 f   jdmarker.obj
 0001:0000827e       _get_soi                   1000927e f   jdmarker.obj
 0001:0000831d       _get_sos                   1000931d f   jdmarker.obj
 0001:00008766       _next_marker               10009766 f   jdmarker.obj
 0001:00008835       _read_markers              10009835 f   jdmarker.obj
 0001:00008a01       $LN100                     10009a01     jdmarker.obj
 0001:00008a0d       $LN99                      10009a0d     jdmarker.obj
 0001:00008a19       $LN102                     10009a19     jdmarker.obj
 0001:00008a3d       $LN101                     10009a3d     jdmarker.obj
 0001:00008a64       _read_restart_marker       10009a64 f   jdmarker.obj
 0001:00008ae3       _reset_marker_reader       10009ae3 f   jdmarker.obj
 0001:00008b11       _save_marker               10009b11 f   jdmarker.obj
 0001:00008d90       _skip_variable             10009d90 f   jdmarker.obj
 0001:00008e30       _finish_output_pass        10009e30 f   jdmaster.obj
 0001:00009064       _master_selection          1000a064 f   jdmaster.obj
 0001:0000929f       _prepare_for_output_pass   1000a29f f   jdmaster.obj
 0001:000093cf       _prepare_range_limit_table 1000a3cf f   jdmaster.obj
 0001:0000944e       _use_merged_upsample       1000a44e f   jdmaster.obj
 0001:000094c9       _build_ycc_rgb_table       1000a4c9 f   jdmerge.obj
 0001:00009582       _h2v1_merged_upsample      1000a582 f   jdmerge.obj
 0001:000096dc       _h2v2_merged_upsample      1000a6dc f   jdmerge.obj
 0001:00009949       _merged_1v_upsample        1000a949 f   jdmerge.obj
 0001:0000997c       _merged_2v_upsample        1000a97c f   jdmerge.obj
 0001:00009a35       _start_pass_merged_upsample 1000aa35 f   jdmerge.obj
 0001:00009a4a       _decode_mcu_AC_first       1000aa4a f   jdphuff.obj
 0001:00009c92       _decode_mcu_AC_refine      1000ac92 f   jdphuff.obj
 0001:0000a086       _decode_mcu_DC_first       1000b086 f   jdphuff.obj
 0001:0000a2b5       _decode_mcu_DC_refine      1000b2b5 f   jdphuff.obj
 0001:0000a3f7       _process_restart           1000b3f7 f   jdphuff.obj
 0001:0000a466       _start_pass_phuff_decoder  1000b466 f   jdphuff.obj
 0001:0000a74e       _post_process_1pass        1000b74e f   jdpostct.obj
 0001:0000a7b2       _post_process_2pass        1000b7b2 f   jdpostct.obj
 0001:0000a84b       _post_process_prepass      1000b84b f   jdpostct.obj
 0001:0000a8f6       _start_pass_dpost          1000b8f6 f   jdpostct.obj
 0001:0000a9a0       _fullsize_upsample         1000b9a0 f   jdsample.obj
 0001:0000a9ab       _h2v1_fancy_upsample       1000b9ab f   jdsample.obj
 0001:0000aa6e       _h2v1_upsample             1000ba6e f   jdsample.obj
 0001:0000aac4       _h2v2_fancy_upsample       1000bac4 f   jdsample.obj
 0001:0000ac01       _h2v2_upsample             1000bc01 f   jdsample.obj
 0001:0000ac6c       _int_upsample              1000bc6c f   jdsample.obj
 0001:0000af35       _noop_upsample             1000bf35 f   jdsample.obj
 0001:0000af3d       _sep_upsample              1000bf3d f   jdsample.obj
 0001:0000b013       _start_pass_upsample       1000c013 f   jdsample.obj
 0001:0000b051       _emit_message              1000c051 f   jerror.obj
 0001:0000b082       _error_exit                1000c082 f   jerror.obj
 0001:0000b097       _format_message            1000c097 f   jerror.obj
 0001:0000b103       _output_message            1000c103 f   jerror.obj
 0001:0000b152       _reset_error_mgr           1000c152 f   jerror.obj
 0001:0000c40d       _access_virt_barray        1000d40d f   jmemmgr.obj
 0001:0000c540       _access_virt_sarray        1000d540 f   jmemmgr.obj
 0001:0000c670       _alloc_barray              1000d670 f   jmemmgr.obj
 0001:0000c72f       _alloc_large               1000d72f f   jmemmgr.obj
 0001:0000c7c3       _alloc_sarray              1000d7c3 f   jmemmgr.obj
 0001:0000c877       _alloc_small               1000d877 f   jmemmgr.obj
 0001:0000c97a       _do_barray_io              1000d97a f   jmemmgr.obj
 0001:0000c9f9       _do_sarray_io              1000d9f9 f   jmemmgr.obj
 0001:0000ca75       _free_pool                 1000da75 f   jmemmgr.obj
 0001:0000cc6d       _out_of_memory             1000dc6d f   jmemmgr.obj
 0001:0000cc8a       _realize_virt_arrays       1000dc8a f   jmemmgr.obj
 0001:0000cdfc       _request_virt_barray       1000ddfc f   jmemmgr.obj
 0001:0000ce64       _request_virt_sarray       1000de64 f   jmemmgr.obj
 0001:0000cecc       _self_destruct             1000decc f   jmemmgr.obj
 0001:0000cf5c       _alloc_fs_workspace        1000df5c f   jquant1.obj
 0001:0000cf9b       _color_quantize            1000df9b f   jquant1.obj
 0001:0000d058       _color_quantize3           1000e058 f   jquant1.obj
 0001:0000d10c       _create_colorindex         1000e10c f   jquant1.obj
 0001:0000d243       _create_colormap           1000e243 f   jquant1.obj
 0001:0000d3b8       _create_odither_tables     1000e3b8 f   jquant1.obj
 0001:0000d511       _new_color_map_1_quant     1000e511 f   jquant1.obj
 0001:0000d525       _quantize3_ord_dither      1000e525 f   jquant1.obj
 0001:0000d663       _quantize_fs_dither        1000e663 f   jquant1.obj
 0001:0000d820       _quantize_ord_dither       1000e820 f   jquant1.obj
 0001:0000d92e       _select_ncolors            1000e92e f   jquant1.obj
 0001:0000da12       _start_pass_1_quant        1000ea12 f   jquant1.obj
 0001:0000dae2       _compute_color             1000eae2 f   jquant2.obj
 0001:0000dc85       _fill_inverse_cmap         1000ec85 f   jquant2.obj
 0001:0000dd90       _find_best_colors          1000ed90 f   jquant2.obj
 0001:0000df23       _find_nearby_colors        1000ef23 f   jquant2.obj
 0001:0000e117       _finish_pass1              1000f117 f   jquant2.obj
 0001:0000e13f       _init_error_limit          1000f13f f   jquant2.obj
 0001:0000e2cd       _median_cut                1000f2cd f   jquant2.obj
 0001:0000e416       _new_color_map_2_quant     1000f416 f   jquant2.obj
 0001:0000e428       _pass2_fs_dither           1000f428 f   jquant2.obj
 0001:0000e750       _pass2_no_dither           1000f750 f   jquant2.obj
 0001:0000e830       _prescan_quantize          1000f830 f   jquant2.obj
 0001:0000e8cc       _select_colors             1000f8cc f   jquant2.obj
 0001:0000e953       _start_pass_2_quant        1000f953 f   jquant2.obj
 0001:0000ea4e       _update_box                1000fa4e f   jquant2.obj
 0001:0000f275       _png_build_16bit_table     10010275 f   png.obj
 0001:0000f40b       _png_build_16to8_table     1001040b f   png.obj
 0001:0000f53a       _png_build_8bit_table      1001053a f   png.obj
 0001:0000fa61       $LN56                      10010a61     png.obj
 0001:0000fa79       $LN55                      10010a79     png.obj
 0001:0000fe0b       _png_fp_sub                10010e0b f   png.obj
 0001:00010897       $LN17                      10011897     png.obj
 0001:00010a1b       _png_default_error         10011a1b f   pngerror.obj
 0001:00010ae6       _png_format_buffer         10011ae6 f   pngerror.obj
 0001:00010f4c       _png_malloc_array_checked  10011f4c f   pngmem.obj
 0001:00011129       _png_do_read_intrapixel    10012129 f   pngread.obj
 0001:000111e7       _png_read_destroy          100121e7 f   pngread.obj
 0001:0001199a       _convert_gamma_value       1001299a f   pngrtran.obj
 0001:00011a0d       _png_do_chop               10012a0d f   pngrtran.obj
 0001:00011a4c       _png_do_compose            10012a4c f   pngrtran.obj
 0001:00012c43       _png_do_encode_alpha       10013c43 f   pngrtran.obj
 0001:00012d00       _png_do_expand             10013d00 f   pngrtran.obj
 0001:00013133       _png_do_expand_16          10014133 f   pngrtran.obj
 0001:00013172       _png_do_expand_palette     10014172 f   pngrtran.obj
 0001:000133e1       _png_do_gamma              100143e1 f   pngrtran.obj
 0001:00013785       _png_do_gray_to_rgb        10014785 f   pngrtran.obj
 0001:00013901       _png_do_quantize           10014901 f   pngrtran.obj
 0001:00013a2a       _png_do_read_filler        10014a2a f   pngrtran.obj
 0001:00013c6d       _png_do_read_invert_alpha  10014c6d f   pngrtran.obj
 0001:00013d18       _png_do_read_swap_alpha    10014d18 f   pngrtran.obj
 0001:000141f4       _png_do_rgb_to_gray        100151f4 f   pngrtran.obj
 0001:00014704       _png_do_scale_16_to_8      10015704 f   pngrtran.obj
 0001:0001475a       _png_do_unpack             1001575a f   pngrtran.obj
 0001:000148ac       _png_do_unshift            100158ac f   pngrtran.obj
 0001:00014a2a       _png_init_gamma_values     10015a2a f   pngrtran.obj
 0001:00014a9b       _png_init_palette_transformations 10015a9b f   pngrtran.obj
 0001:00015569       _png_init_rgb_transformations 10016569 f   pngrtran.obj
 0001:00015830       _png_rtran_ok              10016830 f   pngrtran.obj
 0001:000159ac       _translate_gamma_flags     100169ac f   pngrtran.obj
 0001:000159e7       _unsupported_gamma         100169e7 f   pngrtran.obj
 0001:00015a1c       _png_handle_IHDR           10016a1c f   pngrutil.obj
 0001:00015b6a       _png_handle_PLTE           10016b6a f   pngrutil.obj
 0001:00015cd8       _png_handle_IEND           10016cd8 f   pngrutil.obj
 0001:00015d09       _png_handle_gAMA           10016d09 f   pngrutil.obj
 0001:00015d8d       _png_handle_sBIT           10016d8d f   pngrutil.obj
 0001:00015e90       _png_handle_cHRM           10016e90 f   pngrutil.obj
 0001:0001600c       _png_handle_sRGB           1001700c f   pngrutil.obj
 0001:0001607b       _png_handle_sPLT           1001707b f   pngrutil.obj
 0001:000162ac       _png_handle_tRNS           100172ac f   pngrutil.obj
 0001:00016443       _png_handle_bKGD           10017443 f   pngrutil.obj
 0001:00016610       _png_handle_hIST           10017610 f   pngrutil.obj
 0001:000166f2       _png_handle_pHYs           100176f2 f   pngrutil.obj
 0001:00016789       _png_handle_oFFs           10017789 f   pngrutil.obj
 0001:00016878       _png_handle_pCAL           10017878 f   pngrutil.obj
 0001:00016a57       _png_handle_sCAL           10017a57 f   pngrutil.obj
 0001:00016b94       _png_handle_tIME           10017b94 f   pngrutil.obj
 0001:00016c2c       _png_handle_tEXt           10017c2c f   pngrutil.obj
 0001:00016d32       _png_cache_unknown_chunk   10017d32 f   pngrutil.obj
 0001:00016e00       _png_chunk_index_from_name 10017e00 f   pngrutil.obj
 0001:0001739d       _png_crc_error             1001839d f   pngrutil.obj
 0001:0001743b       _png_crc_finish_critical   1001843b f   pngrutil.obj
 0001:000179d1       _png_get_int_32_checked    100189d1 f   pngrutil.obj
 0001:00017cf6       _png_inflate_claim         10018cf6 f   pngrutil.obj
 0001:00017f71       _png_read_buffer           10018f71 f   pngrutil.obj
 0001:00018121       _png_read_filter_row_avg   10019121 f   pngrutil.obj
 0001:00018174       _png_read_filter_row_paeth_1byte_pixel 10019174 f   pngrutil.obj
 0001:00018216       _png_read_filter_row_paeth_multibyte_pixel 10019216 f   pngrutil.obj
 0001:000182fd       _png_read_filter_row_sub   100192fd f   pngrutil.obj
 0001:0001832b       _png_read_filter_row_up    1001932b f   pngrutil.obj
 0001:00018813       _check_location            10019813 f   pngset.obj
 0001:0001b301       _SplashLoadStream          1001c301 f   splashscreen_impl.obj
 0001:0001b6ae       _closeFile                 1001c6ae f   splashscreen_impl.obj
 0001:0001b6bd       _peekFile                  1001c6bd f   splashscreen_impl.obj
 0001:0001b6e6       _peekMem                   1001c6e6 f   splashscreen_impl.obj
 0001:0001b6fa       _readFile                  1001c6fa f   splashscreen_impl.obj
 0001:0001b715       _readMem                   1001c715 f   splashscreen_impl.obj
 0001:0001b9f4       _my_error_exit             1001c9f4 f   splashscreen_jpeg.obj
 0001:0001ba0f       _set_stream_src            1001ca0f f   splashscreen_jpeg.obj
 0001:0001ba73       _stream_fill_input_buffer  1001ca73 f   splashscreen_jpeg.obj
 0001:0001bade       _stream_init_source        1001cade f   splashscreen_jpeg.obj
 0001:0001baed       _stream_skip_input_data    1001caed f   splashscreen_jpeg.obj
 0001:0001cac9       _SplashWndProc@16          1001dac9 f   splashscreen_sys.obj
 0001:0001d0d0       _bi_flush                  1001e0d0 f   trees.obj
 0001:0001d13c       _bi_windup                 1001e13c f   trees.obj
 0001:0001d193       _build_bl_tree             1001e193 f   trees.obj
 0001:0001d1f9       _build_tree                1001e1f9 f   trees.obj
 0001:0001d473       _compress_block            1001e473 f   trees.obj
 0001:0001d91a       _detect_data_type          1001e91a f   trees.obj
 0001:0001d982       _gen_bitlen                1001e982 f   trees.obj
 0001:0001dba4       _init_block                1001eba4 f   trees.obj
 0001:0001dc13       _pqdownheap                1001ec13 f   trees.obj
 0001:0001dcca       _scan_tree                 1001ecca f   trees.obj
 0001:0001dda6       _send_all_trees            1001eda6 f   trees.obj
 0001:0001dfe8       _send_tree                 1001efe8 f   trees.obj
 0001:0001e9ca       _crc_word                  1001f9ca f   zcrc32.obj
 0001:0001f270       $$000000                   10020270     MSVCRT:ftol2.obj
 0001:0001f28e       L51                        1002028e     MSVCRT:ftol2.obj
 0001:0001f2d3       L52                        100202d3     MSVCRT:ftol2.obj
 0001:0001f2e7       L53                        100202e7     MSVCRT:ftol2.obj
 0001:0001f2e9       L55                        100202e9     MSVCRT:ftol2.obj
 0001:0001f2f3       L56                        100202f3     MSVCRT:ftol2.obj
 0001:0001f30c       L57                        1002030c     MSVCRT:ftol2.obj
 0001:0001f320       $$000000                   10020320     MSVCRT:alloca16.obj
 0001:0001f336       alloca_8                   10020336     MSVCRT:alloca16.obj
 0001:0001f350       ?dllmain_crt_dispatch@@YGHQAUHINSTANCE__@@KQAX@Z 10020350 f   MSVCRT:dll_dllmain.obj
 0001:0001f3a3       ?dllmain_crt_process_attach@@YAHQAUHINSTANCE__@@QAX@Z 100203a3 f   MSVCRT:dll_dllmain.obj
 0001:0001f4aa       ?dllmain_crt_process_detach@@YAH_N@Z 100204aa f   MSVCRT:dll_dllmain.obj
 0001:0001f55a       ?dllmain_dispatch@@YAHQAUHINSTANCE__@@KQAX@Z 1002055a f   MSVCRT:dll_dllmain.obj
 0001:0001f665       ?dllmain_raw@@YGHQAUHINSTANCE__@@KQAX@Z 10020665 f   MSVCRT:dll_dllmain.obj
 0001:0001f890       $$000000                   10020890     MSVCRT:chkstk.obj
 0001:0001f8a4       cs10                       100208a4     MSVCRT:chkstk.obj
 0001:0001f8b2       cs20                       100208b2     MSVCRT:chkstk.obj
 0001:0001f8bb       ___get_entropy             100208bb f   MSVCRT:gs_support.obj
 0001:0001f9aa       ?find_pe_section@@YAPAU_IMAGE_SECTION_HEADER@@QAEI@Z 100209aa f   MSVCRT:utility.obj
 0001:0001fe10       $$000000                   10020e10     MSVCRT:sehprolg4.obj
 0002:000001f0       _configuration_table       100211f0     deflate.obj
 0002:00000268       ?my_version@?1??deflateInit2_@@9@9 10021268     deflate.obj
 0002:00000270       ?CodeMasks@?1??DGifDecompressInput@@9@9 10021270     dgif_lib.obj
 0002:0000028c       ?InterlacedOffset@?9??DGifSlurp@@9@9 1002128c     dgif_lib.obj
 0002:0000029c       ?InterlacedJumps@?9??DGifSlurp@@9@9 1002129c     dgif_lib.obj
 0002:000002c8       ?lenfix@?1??fixedtables@@9@9 100212c8     infback.obj
 0002:00000ac8       ?distfix@?1??fixedtables@@9@9 10021ac8     infback.obj
 0002:00000b48       ?order@?1??inflateBack@@9@9 10021b48     infback.obj
 0002:00000cb0       ?lenfix@?1??fixedtables@@9@9 10021cb0     inflate.obj
 0002:000014b0       ?distfix@?1??fixedtables@@9@9 100224b0     inflate.obj
 0002:00001530       ?order@?1??inflate@@9@9    10022530     inflate.obj
 0002:00001630       ?lbase@?1??inflate_table@@9@9 10022630     inftrees.obj
 0002:00001670       ?lext@?1??inflate_table@@9@9 10022670     inftrees.obj
 0002:000016b0       ?dbase@?1??inflate_table@@9@9 100226b0     inftrees.obj
 0002:000016f0       ?dext@?1??inflate_table@@9@9 100226f0     inftrees.obj
 0002:00001760       ?aanscales@?8??start_pass_fdctmgr@@9@9 10022760     jcdctmgr.obj
 0002:000017e0       ?aanscalefactor@?N@??start_pass_fdctmgr@@9@9 100227e0     jcdctmgr.obj
 0002:00001820       ?std_luminance_quant_tbl@?1??jSetLQuality@@9@9 10022820     jcparam.obj
 0002:00001920       ?std_chrominance_quant_tbl@?1??jSetLQuality@@9@9 10022920     jcparam.obj
 0002:00001a20       ?bits_dc_luminance@?1??std_huff_tables@@9@9 10022a20     jcparam.obj
 0002:00001a34       ?val_dc_luminance@?1??std_huff_tables@@9@9 10022a34     jcparam.obj
 0002:00001a40       ?bits_dc_chrominance@?1??std_huff_tables@@9@9 10022a40     jcparam.obj
 0002:00001a54       ?val_dc_chrominance@?1??std_huff_tables@@9@9 10022a54     jcparam.obj
 0002:00001a60       ?bits_ac_luminance@?1??std_huff_tables@@9@9 10022a60     jcparam.obj
 0002:00001a78       ?val_ac_luminance@?1??std_huff_tables@@9@9 10022a78     jcparam.obj
 0002:00001b1c       ?bits_ac_chrominance@?1??std_huff_tables@@9@9 10022b1c     jcparam.obj
 0002:00001b30       ?val_ac_chrominance@?1??std_huff_tables@@9@9 10022b30     jcparam.obj
 0002:00001bd8       ?aanscales@?L@??start_pass@@9@9 10022bd8     jddctmgr.obj
 0002:00001c58       ?aanscalefactor@?O@??start_pass@@9@9 10022c58     jddctmgr.obj
 0002:00001c98       _extend_test               10022c98     jdhuff.obj
 0002:00001cd8       _extend_offset             10022cd8     jdhuff.obj
 0002:00001d18       _extend_test               10022d18     jdphuff.obj
 0002:00001d58       _extend_offset             10022d58     jdphuff.obj
 0002:00003230       _first_pool_slop           10024230     jmemmgr.obj
 0002:00003238       _extra_pool_slop           10024238     jmemmgr.obj
 0002:00003250       _base_dither_matrix        10024250     jquant1.obj
 0002:00003350       ?RGB_order@?1??select_ncolors@@9@9 10024350     jquant1.obj
 0002:00003ca0       ?png_signature@?1??png_sig_cmp@@9@9 10024ca0     png.obj
 0002:00003ca8       ?short_months@?1??png_convert_to_rfc1123_buffer@@9@9 10024ca8     png.obj
 0002:00004140       ?digits@?2??png_format_number@@9@9 10025140     pngerror.obj
 0002:00004154       ?valid_parameters@?3??png_formatted_warning@@9@9 10025154     pngerror.obj
 0002:00004160       _png_digit                 10025160     pngerror.obj
 0002:00004258       _png_pass_start            10025258     pngpread.obj
 0002:00004260       _png_pass_inc              10025260     pngpread.obj
 0002:00004268       _png_pass_ystart           10025268     pngpread.obj
 0002:00004270       _png_pass_yinc             10025270     pngpread.obj
 0002:0000431c       ?sRGB_xy@?1??chromaticities_match_sRGB@@9@9 1002531c     pngread.obj
 0002:0000433c       ?chunks_to_process@?2??png_image_skip_unused_chunks@@9@9 1002533c     pngread.obj
 0002:00004718       _png_pass_start            10025718     pngrutil.obj
 0002:00004720       _png_pass_inc              10025720     pngrutil.obj
 0002:00004728       _png_pass_ystart           10025728     pngrutil.obj
 0002:00004730       _png_pass_yinc             10025730     pngrutil.obj
 0002:00004738       _read_chunks               10025738     pngrutil.obj
 0002:00004818       ?row_mask@?4??png_combine_row@@9@9 10025818     pngrutil.obj
 0002:000048a8       ?display_mask@?4??png_combine_row@@9@9 100258a8     pngrutil.obj
 0002:00004d60       ?chunks_to_ignore@?4??png_set_keep_unknown_chunks@@9@9 10025d60     pngset.obj
 0002:00005120       _onebppswaptable           10026120     pngtrans.obj
 0002:00005220       _twobppswaptable           10026220     pngtrans.obj
 0002:00005320       _fourbppswaptable          10026320     pngtrans.obj
 0002:00005548       ?scale@?1??quantizeColors@@9@9 10026548     splashscreen_gfx_impl.obj
 0002:00005554       _szNetscape20ext           10026554     splashscreen_gif.obj
 0002:00005560       _formats                   10026560     splashscreen_impl.obj
 0002:00005900       _extra_lbits               10026900     trees.obj
 0002:00005978       _extra_dbits               10026978     trees.obj
 0002:000059f0       _extra_blbits              100269f0     trees.obj
 0002:00005a3c       _bl_order                  10026a3c     trees.obj
 0002:00005a50       _static_ltree              10026a50     trees.obj
 0002:00005ed0       _static_dtree              10026ed0     trees.obj
 0002:00005f48       _base_length               10026f48     trees.obj
 0002:00005fc0       _base_dist                 10026fc0     trees.obj
 0002:00006038       _static_l_desc             10027038     trees.obj
 0002:0000604c       _static_d_desc             1002704c     trees.obj
 0002:00006060       _static_bl_desc            10027060     trees.obj
 0002:00006078       _crc_table                 10027078     zcrc32.obj
 0002:00006478       _crc_big_table             10027478     zcrc32.obj
 0002:00006878       _crc_braid_table           10027878     zcrc32.obj
 0002:00007878       _crc_braid_big_table       10028878     zcrc32.obj
 0002:00008878       _x2n_table                 10029878     zcrc32.obj
 0002:000089f0       _GS_ExceptionPointers      100299f0     MSVCRT:gs_report.obj
 0002:00008a00       two32                      10029a00     MSVCRT:ftol2.obj
 0002:00008a04       two63                      10029a04     MSVCRT:ftol2.obj
 0002:00008a08       _NaN                       10029a08     MSVCRT:ftol2.obj
 0002:00008a10       _bias_low                  10029a10     MSVCRT:ftol3.obj
 0002:00008a20       _bias_high                 10029a20     MSVCRT:ftol3.obj
 0002:00008a30       _DP2to32                   10029a30     MSVCRT:ftol3.obj
 0002:00008a38       _NaN                       10029a38     MSVCRT:ftol3.obj
 0002:00008a3c       _onept5                    10029a3c     MSVCRT:ftol3.obj
 0002:00008f68       __sehtable$?dllmain_crt_process_attach@@YAHQAUHINSTANCE__@@QAX@Z 10029f68     MSVCRT:dll_dllmain.obj
 0002:00008f88       __sehtable$?dllmain_crt_process_detach@@YAH_N@Z 10029f88     MSVCRT:dll_dllmain.obj
 0002:00008fb0       __sehtable$?dllmain_dispatch@@YAHQAUHINSTANCE__@@KQAX@Z 10029fb0     MSVCRT:dll_dllmain.obj
 0002:00008fd0       __sehtable$___scrt_is_nonwritable_in_current_image 10029fd0     MSVCRT:utility.obj
 0002:00009340       .edata                     1002a340     splashscreen.exp
 0002:00009368       rgpv                       1002a368     splashscreen.exp
 0002:000093b0       rgszName                   1002a3b0     splashscreen.exp
 0002:000093f8       rgwOrd                     1002a3f8     splashscreen.exp
 0002:0000941c       szName                     1002a41c     splashscreen.exp
 0002:0000942d       $N00001                    1002a42d     splashscreen.exp
 0002:0000943b       $N00002                    1002a43b     splashscreen.exp
 0002:00009462       $N00003                    1002a462     splashscreen.exp
 0002:0000948d       $N00004                    1002a48d     splashscreen.exp
 0002:000094bf       $N00005                    1002a4bf     splashscreen.exp
 0002:000094f0       $N00006                    1002a4f0     splashscreen.exp
 0002:0000951c       $N00007                    1002a51c     splashscreen.exp
 0002:0000954c       $N00008                    1002a54c     splashscreen.exp
 0002:00009577       $N00009                    1002a577     splashscreen.exp
 0002:000095a5       $N00010                    1002a5a5     splashscreen.exp
 0002:000095cd       $N00011                    1002a5cd     splashscreen.exp
 0002:000095d9       $N00012                    1002a5d9     splashscreen.exp
 0002:000095f2       $N00013                    1002a5f2     splashscreen.exp
 0002:00009615       $N00014                    1002a615     splashscreen.exp
 0002:00009620       $N00015                    1002a620     splashscreen.exp
 0002:0000962f       $N00016                    1002a62f     splashscreen.exp
 0002:00009640       $N00017                    1002a640     splashscreen.exp
 0002:00009655       $N00018                    1002a655     splashscreen.exp
 0002:00009974       .idata$6                   1002a974     kernel32:KERNEL32.dll
 0002:00009a5a       .idata$6                   1002aa5a     gdi32:GDI32.dll
 0002:00009a7c       .idata$6                   1002aa7c     java:java.dll
 0002:00009afe       .idata$6                   1002aafe     vcruntime:VCRUNTIME140.dll
 0002:00009cc4       .idata$6                   1002acc4     ucrt:api-ms-win-crt-stdio-l1-1-0.dll
 0002:00009ce4       .idata$6                   1002ace4     ucrt:api-ms-win-crt-heap-l1-1-0.dll
 0002:00009d04       .idata$6                   1002ad04     ucrt:api-ms-win-crt-string-l1-1-0.dll
 0002:00009d26       .idata$6                   1002ad26     ucrt:api-ms-win-crt-convert-l1-1-0.dll
 0002:00009d48       .idata$6                   1002ad48     ucrt:api-ms-win-crt-runtime-l1-1-0.dll
 0002:00009d6a       .idata$6                   1002ad6a     ucrt:api-ms-win-crt-environment-l1-1-0.dll
 0002:00009d90       .idata$6                   1002ad90     ucrt:api-ms-win-crt-math-l1-1-0.dll
 0003:00000000       ?scale@?1??GetScreenDpi@@9@4MA 1002b000     systemScale.obj
 0003:000000b8       ?clazz@?1??Java_java_awt_SplashScreen__1getBounds@@9@9 1002b0b8     java_awt_SplashScreen.obj
 0003:000000bc       ?mid@?1??Java_java_awt_SplashScreen__1getBounds@@9@9 1002b0bc     java_awt_SplashScreen.obj
 0003:000000c4       ?preInitialized@?1??SplashGetInstance@@9@9 1002b0c4     splashscreen_impl.obj
 0003:000000c8       ?splash@?1??SplashGetInstance@@9@9 1002b0c8     splashscreen_impl.obj
 0003:00002e38       ?hLibSHCoreDll@?1??GetScreenDpi@@9@4PAUHINSTANCE__@@A 1002de38     systemScale.obj
 0003:00002e3c       ?lpGetDpiForMonitor@?1??GetScreenDpi@@9@4P6GJPAUHMONITOR__@@HPAI1@ZA 1002de3c     systemScale.obj
 0003:00002e60       _GS_ExceptionRecord        1002de60     MSVCRT:gs_report.obj
 0003:00002eb0       _GS_ContextRecord          1002deb0     MSVCRT:gs_report.obj
 0003:0000317c       ?__proc_attached@@3HA      1002e17c     MSVCRT:dll_dllmain.obj
 0003:00003198       ?is_initialized_as_dll@@3_NA 1002e198     MSVCRT:utility.obj
 0003:00003199       ?module_local_atexit_table_initialized@@3_NA 1002e199     MSVCRT:utility.obj
 0003:0000319c       ?module_local_atexit_table@@3U_onexit_table_t@@A 1002e19c     MSVCRT:utility.obj
 0003:000031a8       ?module_local_at_quick_exit_table@@3U_onexit_table_t@@A 1002e1a8     MSVCRT:utility.obj
 0004:00000060       $R000000                   1002f060     splashscreen.dll.res
